:1072BA00758400852ED2852FD3E4F52FF52E30382C
:1072CA0010E50D852DF0A4252EF52EE5F0352FF5C8
:1072DA002F229072F6303E031272E622E50E251B2B
:1072EA00F50EE51F351AF51F93F50D227F82858865
:1072FA008C8F9295989B9EA1A4A7AAADB0B3B6B95C
:10730A00BBBEC1C3C6C9CBCED0D3D5D7D9DCDEE08C
:10731A00E2E4E6E7E9EBEDEEF0F1F2F4F5F6F7F880
:10732A00F9FAFBFCFCFDFDFEFEFEFEFEFEFEFEFE85
:10733A00FEFDFDFCFCFBFAFAF9F8F7F6F4F3F2F0BD
:10734A00EFEDECEAE8E7E5E3E1DFDDDBD8D6D4D11F
:10735A00CFCDCAC8C5C2C0BDBAB7B4B2AFACA9A670
:10736A00A3A09D9A9794908D8A8784817E7A777458
:10737A00716E6B6865625F5C595653504D4A47445B
:10738A00423F3C393734322F2D2A282624211F1D0B
:10739A001B1918161412110F0E0C0B0A08070605F2
:1073AA0004040302020101000000000000000000C2
:1073BA000001010202030405060708090A0B0D0E63
:1073CA001011131516181A1C1E20222427292B2ED9
:1073DA00303335383A3D404245484B4E5154565960
:0C73EA005C606366696C6F7275787B7F75
:10788F00D2F4C2F5C2F675840F85F0C812781A7457
:10789F00031278DE12780A74031278DE1277F91267
:1078AF0077F974031278DE1277F974021278DE1208
:1078BF0077F9742812794A740612794A740E12797C
:1078CF004A740112794A12780A748012794A22C0D6
:1078DF0000A2E092F3A2E192F2A2E292F1A2E3926D
:1078EF00F0D2F475840F85F0C8C2F47830D8FE85D5
:1078FF00F0C87830D8FED00022C00075840FA2E403
:10790F0092F3A2E592F2A2E692F1A2E792F0D2F4FC
:10791F0085F0C8C2F47830D8FE85F0C87830D8FE2C
:10792F00D00022EF75840FD2F5C2F685F0C8127918
:10793F00081277F91278DE1277F92275840FC2F5E3
:10794F00C2F685F0C81279081277F91278DE12772D
:10795F00F922EF14A2E492E6C2E4D2E712794A22A6
:10796F00740F12794A22740D12794A227F0112790B
:10797F006178107F20127932D8F9227F1112796144
:0A798F0078107F20127932D8F92217
:10717D00C293758400D2C2C2C6D2C6C2C4D2C5C221
:10718D00C330C3FD74A0F5C2C2C5C2C330C3FD8EEA
:10719D00C2C2C330C3FD8FC2C2C330C3FD8DC2C2D4
:1071AD00C330C3FDD2C4C2C320C4FD12780AD2932A
:1071BD0022758400C2C3D2C530C3FD74A0F5C2C20E
:1071CD00C5C2C330C3FD8EC2C2C330C3FD8FC2C2A0
:1071DD00C330C3FDC2C4D2C5C2C330C3FD74A1F553
:1071ED00C2C2C5C2C330C3FDC2C2C2C330C3FD8556
:1071FD00C207D2C4C2C320C4FD22D2C2C2C6D2C6E7
:10720D00D2C4C2C320C4FD22C293758400D2C2C2AF
:10721D00C6D2C6C2C4D2C5C2C330C3FD74A0F5C2A6
:10722D00C2C5C2C330C3FD8EC2C2C330C3FD8FC23F
:10723D00C2C330C3FD8C838D827B80E0A3F5C2C2B7
:10724D00C330C3FDDBF5D2C4C2C320C4FD12780A1E
:10725D00D29322758400C2C3D2C530C3FD74A0F58C
:10726D00C2C2C5C2C330C3FD8EC2C2C330C3FD8FFF
:10727D00C2C2C330C3FDC2C4D2C5C2C330C3FD74C4
:10728D00A1F5C2C2C5C2C330C3FD8C838D82C2C3FA
:10729D0030C3FDE5C2F0A31BBB01F3C2C2C2C330B4
:0D72AD00C3FDE5C2F0D2C4C2C320C4FD225F
:030003000257A3FE
:01000B0032C2
:030013000273F67F
:01001B0032B2
:1063490075FF0775FFDE75FFAD75840F75E107757C
:10635900E21475E34475840F75A48D75A50875A6B7
:106369000075A7FF759CFF759D00759ECC759FF8FC
:1063790075A0FF75B00075C80075D8FF75E833754D
:10638900F80775AD0F75840175893075888F758427
:106399000275893075888F75840F758A80758C6749
:1063A900780874FF000000000000000000000000F1
:1063B900D5E0F1D8EDE58C30E7FB759701758A00DA
:1063C90043890475840075B71075840F4389017575
:1063D9008D02758F01758E047480D5E0FD438902A5
:1063E900E58930E4FB75970275840075D1077584DA
:1063F9000075BB0175BA0075BCF075C70075C6009C
:1064090075C5FF75C4FF75E80075840275BB047511
:10641900BA0075BCF175C60075C4FF75E88075844E
:106429000075D48475840175D484758400C2F875A7
:106439009A47759D1A75F80175870075840075B9B5
:106449000075A9007591007598507584017598902B
:1064590075840075C04075C30075CFC97584007512
:106469008E10758921758805758400758A00758B6C
:10647900E0758CF4758DE043884075840075C9001A
:1064890075CA0075CB0075CC0075CD007584017592
:10649900C91875CA8075CBFB75CDFB75CC80D2CA7E
:1064A90075840275C91875CAA675CBAF75CDAF7558
:1064B900CCA6D2CA75840075EF0275A8AC75B83D33
:1064C90075E6B075E71575F60075F741789E760A99
:0864D900769F780A78A0760690
:1064E10075A8959000007F007E20E4F0A3DFFCDE1C
:1064F100FA789E760A789F760A78A07606D2937506
:06650100E8FF1272072200
:1077730075840FD2FD2275840FC2FD22E490FC00B4
:10778300732275840FD2EA2275840FC2EA227584AC
:107793000FA2EC2275840FD2FE2275840FC2FE2243
:1077A30075840FC2FF2275840FD2FF2275840FA246
:1077B300FA2275840FA2F92275840FA2DD22A29208
:1077C3002275840FA2DA2275840FA2DB2275840F3F
:1077D300A2D82275840FA2D9220000000000000065
:1077E3000000000000000000000000000000000096
:1077F300000000000022C000C001790878B4D8FE60
:10780300D9FAD001D00022C000C0E0789A7605E60C
:1078130070FDD0E0D00022C000C0E0789A760FE679
:1078230070FDD0E0D00022EF75F064842430900026
:107833005EF0E5F0A375F00A842430F0A3E5F024AC
:1078430030F022EF75F06484243090005EF0E5F0B0
:10785300A375F00A842430F0A3E5F02430F09000FF
:097863005EE0B4300B7420F0A3C8
:10786C00E0B430037420F02275F06484F6E5F0087F
:10787C0075F00A84F608A6F00822850607222285F0
:03788C00050622CC
:1057A300758400C2CA85CC3A85CD3975CC0075CDD8
:1057B30000D2CA10CF02D25B32305B0BC25BE53939
:1057C300C394364002800122788F798D7B06E7F6F9
:1057D3001819DBFAA63918A63AAA3AAB39AE02AFC2
:1057E30003EEC4035407FEEFC403FF54F84EFEEF69
:1057F3005407FF7803798AC3E79AFC09E79BFD09FD
:1058030050066304FF6305FFC3EC9EED9F5074D8FD
:10581300E6789779957C06E7F61819DCFAA603185B
:10582300A6027992AE02AF03EEC423541FFEEFC467
:1058330023FF54E04EFEEF541FFF7803C3E79AFCA7
:1058430009E79BFD0950066304FF6305FFC3EC9E54
:10585300ED9F502FD8E678907A007B007C00790486
:10586300EA26FA08EB36FB08EC3400FCD9F2EC1319
:0D587300FCEB13FBEA13FAEC13EB13F53812
:10588000EA13F537D23A22303A31C23A1258BC50B4
:105890002A853E3F853D3E853C3D853B3C85073B1B
:1058A000303913E5416F600EE507B53C0EB53D0B91
:1058B000B53E08B53F05850740D23B229059D7E554
:1058C0003893FF90590323232582F582E583340022
:1058D000F5831258E2400A0F1258E240040F1258A2
:1058E000E222E493F9A3E493FAA3E493FBA3E49301
:1058F000FCA3C3E5379AE538995007C3EC9537EB1D
:10590000953822EA25DD89DD89D324D324CBD2CB77
:10591000D2C4DBC4DBBE39BE39B7CAB7CAB18EB197
:105920008EAB87AB87A59CA59CA000A0009A969AF9
:105930009695D895D891E591E58D858D8588AF8828
:10594000AF840C840C7F9A7F9A7B497B49771B77C5
:105950001B730F730F6F276F276B576B5767AB67FF
:10596000AB642C642C60C660C65D795D795AFE5AC2
:10597000FE5970597057E257E25661566154E75428
:10598000E7537453745207520750A050A04F404F32
:10599000404DE64DE64C934C934B414B4149F54904
:1059A000F548B548B547764776463E463E450845F4
:1059B00008432A432A40E440E43F533F533E3E3EDF
:1059C0003E3C943C943A863A86391839183805009A
:1059D0000000000000000032323232323232323205
:1059E0003232323232323232323232323232323297
:1059F0003232323232323232323232323232323287
:105A00003232323232323232323232323232323276
:105A1000313130302F2E2D2D2D2C2C2B2A292928B9
:105A200027262525242323222120201F1E1E1D1C5E
:105A30001C1B1A1A1A1A19191918181817171717D8
:105A4000161616161515151514141414131313130E
:105A5000121212121111111110101010100F0F0F3D
:105A60000F0F0E0E0E0E0D0D0D0D0C0C0C0C0B0B66
:105A70000B0B0B0B0A0A0A0A0A090909090909088A
:105A800008080808080707070707070606060606A6
:105A900006060505050505050404040404040403BD
:105AA00003030303030302020202020202010101D3
:105AB00001010101010101010101010000000000DB
:105AC00000000000000000000000000000000000D6
:075AD00000000000000000CF
:106D9200C007C0007F011279617F4C1279327F54A3
:106DA2001279327F521279327F20127932204904CD
:106DB2007F3080027F311279327F20127932900146
:106DC200EAE0784D12787C784D86074307301279D5
:106DD200320886074307301279327507201279325A
:106DE2009001EBE0784D127874784D8607430730B6
:106DF2001279320886074307301279320886074330
:106E020007301279327507201279329001ECE0785E
:106E12004D12787C784D8607430730127932088606
:106E220007430730127932750720127932D000D029
:106E32000722C007C0007F111279617F4C1279329C
:106E4200750720127932204E047F3080027F311282
:106E520079327F201279329001B4E0784D12787C39
:106E6200784D860743073012793208860743073088
:106E72001279327507201279329001B5E0784D12FD
:106E82007874784D860743073012793208860743B3
:106E920007301279320886074307301279327507B4
:106EA200201279329001B6E0784D12787C784D86C6
:106EB20007430730127932088607430730127932C6
:106EC2007507201279329001B7E0784D12787C78FC
:106ED2004D8607430730127932088607430730127E
:076EE2007932D000D0072235
:106AD500003800512372461765340E5F2D7C481926
:106AE5006B3A1C4D3F6E5A0B7928124331605405A1
:106AF5007726001F3D227A654758756A48570F105B
:106B0500322D6877554A120D2F301D02203F6778C8
:106B15005A45006245270B694E2C157750321E7C6D
:106B25005B39294B6C0E224067053C5E791B375556
:106B3500721052301775593B1C7E472502604C2E4A
:106B4500096B7B193E5C701235576E0C2B49650736
:106B55002042264463012D4F680A33517614385A72
:106B65007D1F0F6D4A28046641231A785F3D117316
:106B75005436741631537F1D3A58610324466A080A
:106B85002F4D5D3F187A56341371482A0D6F4321F6
:106B950006644F2D0A68442601635A381F7D513318
:106BA5001476660423416D0F284A73113654781AFA
:106BB5003D5F1D7F583A16745331086A4D2F0361A6
:106BC5004624345671133F5D7A18214364062A48DA
:106BD5006F0D690B2C4E620027457C1E395B7715BE
:106BE5003250402205674B290E6C553710725E3CBA
:106BF5001B793B597E1C305275172E4C6B09254766
:106C0500600212705735197B5C3E076542200C6E99
:106C1500492B004307440D4E0A49195A1E5D145766
:106C25001350317236753C7F3B78286B2F6C256687
:026C35002261DA
:107E6200788376ACA24EE433FFC4333354C0FE9021
:107E720001B6E0FD541F25E04EFE9001B4E0FC5433
:107E820010C4540F4E7882F6EC540FC454F0FE9096
:107E920001B5E0FC54F0C4540F4E7881F6EC540F57
:107EA200C454F0FE9001B7E0FC541EC3134E788018
:107EB200F6EF3395E0FE74D52FF582746A3EF583B2
:107EC200E493FFED906AD793FEEF6EFF9001B4E06A
:107ED200906AF7936FFF9001B5E0906B17936FFF75
:107EE200EC906C17936F787FF69001B7E030E00466
:0B7EF200E64480F6D257787E76282206
:1088F000758401309915C299205110D251759898FC
:10890000D29C78987604900243800F309846209A43
:108910000DE5997009C298900244740FF0229001FD
:10892000B3E06401702CE54B75F0058420551024EC
:1089300049F582E43401F583E599F0D2558010249D
:108940005EF582E43401F583E599F0C255D256C252
:058950009822C29822EC
:107A9600758401309902C299209803027B7620539F
:107AA60017209A11E599700DD253754C0AF54B9033
:107AB6000243740FF0C29822209A0FE599700B903A
:107AC6000243740FF090024480739001B3E0FF64A8
:107AD60001702CE54B75F005842055102449F5827C
:107AE600E43401F583E599F0D2558010245EF582E1
:107AF600E43401F583E599F0C255D256C29822EFD7
:107B0600B4021AAB550557E557AA56700205561426
:107B1600F9E59912853C9001B3740380209001B376
:107B2600E0FFB4031CAB550557E557AA567002058E
:107B36005614F9E59912853C9001B37404F0C29885
:107B460022EFB404299001E5E0FF04F074BC2FF5A0
:107B560082E43401F583E599F0C2989001E5E0B43A
:107B6600280E9001E77401F0E49001B3F022C29868
:017B760022EC
:109132002052221277A943E740754C0AE4F54B907E
:1091420001B3F0C2519001FBF0D2527584017598BF
:0691520090C29CF5992279
:108955009001E6E0705C90020BE0FF7025D390017A
:10896500B9E094869001B8E094674008E4F0A374F8
:1089750002F0800E9001B9E02428F09001B8E034AF
:1089850000F09001B9E02FFF9001B8E03400FE122D
:1089950071BE90020BE024BCF582E43401F583EF4F
:1089A500F090020BE004F0E0B42807E4F09001E653
:0389B50004F022A9
:10802E009001E7E070030280BF9001BAE0FEA3E08A
:10803E00FF4E6009C3EF9402EE94005006E49001E7
:10804E00E7F02290020BE0FF9001BBE02FFF9001C2
:10805E00BAE03400FE1271BE90020BE024BCF58231
:10806E00E43401F583E0FD6F601790020BE0FF90A2
:10807E0001BBE02FFF9001BAE03400FE12717DD2F9
:10808E005490020BE004F0E0B42826E49001E7F0EF
:10809E0090020BF09001BAE07004A3E0640270113C
:1080AE0030540EC254127EFD1289B8128A14126117
:0280BE0054224A
:108755003051647584019001FBE0B40D00505590D3
:10876500876BF828287302879202879502879802FB
:10877500879B02879E0287A10287A40287A702879B
:10878500AA0287AD0287B00287B30287B602915865
:1087950002933D028E0E028E8202922902005E0233
:1087A5008FCC020026028EBA028D5602929A029151
:0887B500090292B11292F322B5
:109158007898E67020759898754C0AF54B9001B38D
:10916800F0900065E09001FBB401047404F022E083
:0691780004F01277A322AF
:0F933D009001B37401F0C2559001FBE004F022DF
:108E0E00900065E01475F005A4B54B15E4B5F011AE
:108E1E007598981277A9E49001B3F09001FB740451
:108E2E00F0E54B75F00584AFF0BF010EC256900110
:0B8E3E00B37401F09001FBE004F0228F
:108E8200E54B75F00584AFF0BF042C20561EE54B70
:108E920075F00584FF2449F582E43401F583E4F09A
:108EA200745E2FF582E43401F583E4F0E49001B3BB
:088EB200F09001FBE014F02236
:10922900900065E075F005A424FDB54B1190005C34
:0F923900E0F599E49001B3F09001FBE004F0221E
:0D005E0090005DE0F5999001FBE004F022B8
:108FCC00900065E0FD75F005A4FFE54BB5071FE4C7
:108FDC00B5F01BEDB414079001FB7409F022127765
:0F8FEC00A3C255E49001B3F09001FBE004F02222
:10002600E54BB4640E1277A9E49001B3F09001FB9E
:100036007409F0E54B75F00584AFF0BF010EC256AA
:0D0046009001B37401F09001FBE004F02282
:108EBA00E54B75F00584AFF0BF042C20561EE54B38
:108ECA0075F00584FF2449F582E43401F583E4F062
:108EDA00745E2FF582E43401F583E4F0E49001B383
:088EEA00F09001FBE014F022FE
:108D5600E54BB465389001E6E0B4012B7555017515
:108D660056017557B8E49001B3F0758401AB55050B
:108D760057E557AA567002055614F91284F6F59966
:0E8D86009001FBE004F0229001FB740CF0223F
:10929A00AB55AA56A9571284F6F599E49001E4F061
:0792AA009001FBE004F0223B
:109109009001E4E0FF04F074BC2FF582E43401F52A
:1091190083E0F5999001E4E0D39428400BE49001B1
:09912900E6F09001FBE004F022E5
:1092B100E54BB46911C251C252E4900147F09001EB
:0792C100B3F09001FBF02265
:1092F300C251C252E4F54B900147F09001B3F09094
:0493030001FBF02258
:108AC9003053527584019001FCE0B40A0050439080
:108AD9008ADFF8282873028AFD028B00028B0302C1
:108AE9008B06028B09028B0C028B0F028B12028BF5
:108AF90015028B18028FFB028E49028EF2029266D2
:108B09000200760290B1028D15028F2A0291C902E4
:068B1900932C12009622CD
:108FFB00E54B7029759898900065E0B4010F1277D6
:10900B00A9E49001B3F09001FC7403F0221277A352
:0E901B00C255E49001B3F09001FCE004F02295
:108E4900900065E01475F005A4B54B11E4B5F00D7B
:108E59007598981277A99001FC7403F022E54B7577
:108E6900F00584AFF0BF0110C256C2559001B3742A
:098E790001F09001FCE004F0227C
:108EF200E54B75F00584AFF0BF042C20561EE54B00
:108F020075F00584FF2449F582E43401F583E4F029
:108F1200745E2FF582E43401F583E4F0E49001B34A
:088F2200F09001FCE014F022C4
:10926600900065E075F005A424FDB54B0E90005CFA
:0C927600E0F599C2559001FCE004F022E4
:0D00760090005DE0F5999001FCE004F0229F
:1090B100900065E0FFB414079001FC7406F022EF04
:1090C10075F005A4B54B14E4B5F0101277A3900127
:0C90D100FCE004F0C255E49001B3F02272
:108D1500E54B75F00584AFF0BF0111C256C2559001
:108D250001B37401F09001FCE004F022E54BB4645A
:108D35001F1277A39001E7E0700B9001B3F090014B
:108D4500FC7408F022E49001B3F09001FC7409F082
:018D550022FB
:108F2A00E54B75F00584AFF0BF042C20561EE54BC7
:108F3A0075F00584FF2449F582E43401F583E4F0F1
:108F4A00745E2FF582E43401F583E4F0E49001B312
:088F5A00F09001FCE014F0228C
:1091C900E54BB4651A7555017556017557BAE490A2
:1091D90001E5F09001FC7409F09001B37402F022EA
:10932C00E54BB4690BC253E49001B3F09001FCF02F
:01933C00220E
:0C009600C253E49001B3F09001FCF02292
:10765500789BE6600116900000E0600214F090004F
:1076650001E0600214F0900002E0600214F0900066
:107675000CE0600214F090000AE0600214F0900043
:107685000DE0600214F090000BE0600214F090022F
:1076950043E0600214F0900244E0600214F09002AE
:1076A5000CE0600214F0789D16E6600302777278AC
:1076B5009D760A789CE6600116900004E06002144D
:1076C500F0900005E0600214F0900006E0600214FE
:1076D500F0900008E0600214F0900009E0600214E8
:1076E500F078A1E6600116900003E0600214F090C6
:1076F500024CE0600214F0900205E0600214F09084
:107705000222E0600214F0789E16E67060789E769C
:107715000A900010E0600214F090000EE07002A3E1
:10772500E0600E90000FE024FFF090000EE034FFC3
:10773500F09001FEE0600214F0900200E060021497
:10774500F0900204E0600214F0900206E06002147A
:10775500F0789F16E67016789F760A78A016E67080
:0E7765000C78A07606900203E0600214F02279
:1092DE00C2B59000037405F0900003E06004C2B5BF
:0592EE0080F6D2B5225C
:10882400535155452020434F53202053454E534523
:10883400004F4E20202020202020202020202020F7
:1088440020004F46462020202020202020202020C9
:10885400202000534954453A20202020525054529D
:108864003A2020002044535020425553205265732F
:1088740065742020002020454570726F6D2077724A
:068884006F6E6721200069
:1091A400757901E579C394155018AF7974722FF568
:1091B40082E43401F583E0FFEF60037F0122057947
:0491C40080E17F00C7
:0191C8002284
:108A7000205755127C45EF6401704D9000A4E0FF33
:108A8000EF24FF924E9001B2E0FF749C2FF582E438
:108A90003401F583E0FF9001B4EFF09001B2E0FF04
:108AA00074872FF582E43401F583E0FF9001B5EF80
:108AB000F09001B2E0FF9001B6EFF012826E9001EB
:098AC000B7EFF0127E62D23F22F2
:107C4500900142E4F0A3E4F0900145E4F0A3E4F0F0
:107C5500900141E4F0900141E0FFEFC3941540032A
:107C6500027CE99001B2E0FFEFD394144006900145
:107C7500B27401F09001B2E0FF74722FF582E43422
:107C850001F583E0FF900144EFF0900144E0FFEF40
:107C9500B401159001B2E0FF74722FF582E434014E
:107CA500F5837402F07F0122900144E0FFEFB402F6
:107CB50024900142E0FEA3E0FFEF4E7018900142D0
:107CC500E4F0A37401F09001B2E0FF7E009001455D
:107CD500EEF0A3EFF09001B2E004F0900141E00472
:107CE500F0027C5A900142E0FEA3E0FFEF4E7004E3
:107CF5007F002222900146E0FF9001B2EFF07F0164
:017D0500225B
:107B7700900142E4F0A3E4F0900145E4F0A3E4F0BF
:107B8700900141E4F0900141E0FFEFC394154003F9
:107B9700027C289001B2E0FFEFD3941440069001D5
:107BA700B27401F09001B2E0FF74722FF582E434F1
:107BB70001F583E0FF900144EFF0900144E0FFEF0F
:107BC7006050900065E0FF9001B2E0FEEE6F60420A
:107BD700900144E0FFEFB401159001B2E0FF747229
:107BE7002FF582E43401F5837402F07F01229001BE
:107BF70042E0FEA3E0FFEF4E70189001B2E0FF7E77
:107C070000900145EEF0A3EFF0900142E4F0A37479
:107C170001F09001B2E004F0900141E004F0027B32
:107C27008C900142E0FEA3E0FFEF4E70047F00223C
:0E7C370022900146E0FF9001B2EFF07F0122A3
:10826E00900065E0FF74482FF582E43401F583E059
:10827E00FFEFB4FF06900065E0FF22757A00E57A05
:10828E00C39414505BAF7AEF25E024F2F582E43408
:10829E0000F583E0FF900065E0FE74C82EF582E4E1
:1082AE003400F583E0FEEEC39F4031AF7AEF25E058
:1082BE0024F1F582E43400F583E0FF74482FF58253
:1082CE00E43401F583E0FFEFB4FF11AF7AEF25E060
:1082DE0024F1F582E43400F583E0FF22057A809ED6
:0282EE007F000F
:0182F000226B
:10837400757B00E57BC394145074AF7BEF25E02438
:10838400F2F582E43400F583E0FF900065E0FE74CA
:10839400C82EF582E43400F583E0FEEEC39F404A24
:1083A400AF7BEF25E024F1F582E43400F583E0FFB0
:1083B40074482FF582E43401F583E0FFEFB4FF2A1B
:1083C400AF7BEF25E024F1F582E43400F583E0FF90
:1083D400900065E0FEEF6E6011AF7BEF25E024F1C5
:1083E400F582E43400F583E0FF22057B80857F007D
:0183F4002266
:1083F500757C00E57CC394145074AF7CEF25E024B4
:108405001AF582E43401F583E0FF900065E0FE741F
:10841500C82EF582E43400F583E0FEEEC39F404AA2
:10842500AF7CEF25E02419F582E43401F583E0FF04
:1084350074482FF582E43401F583E0FFEFB4FF2A99
:10844500AF7CEF25E02419F582E43401F583E0FFE4
:10845500900065E0FEEF6E6011AF7CEF25E024191A
:10846500F582E43401F583E0FF22057C80857F00F9
:0184750022E4
:06001C00900065E0FF22E8
:107527009001B1E0FFEFD3941440069001B17401CC
:10753700F0900141E4F09001B1E0FF74872FF582EC
:10754700E43401F583E0FF9001B1E0FE745D2EF5B0
:1075570082E43401F583E0FEEEB507269001B1E041
:10756700FF749C2FF582E43401F583E0FF9001B1AD
:10757700E0FE74482EF582E43401F583E0FEEE6FF9
:1075870060069001417401F09001B1E0FF74482F4B
:10759700F582E43401F583E0FF900065E0FEEF6ECD
:1075A700600E900065E0FF9001B1E0FEEE6F703A6B
:1075B700900141E0FFEF60439001B1E0FFEFD3940A
:1075C7001550149001B1E0FF74722FF582E4340175
:1075D700F5837401F080249001B1E0FF74722FF5F8
:1075E70082E43401F583E4F080119001B1E0FF7487
:1075F700722FF582E43401F583E4F0900141E0FF56
:10760700EF60449001B1E0FF745D2FF582E434012F
:10761700F583E0FF9001B1E0FE74872EF582E43434
:1076270001F583EFF09001B1E0FF74482FF582E494
:107637003401F583E0FF9001B1E0FE749C2EF582E2
:0E764700E43401F583EFF09001B1E004F0228D
:106C37009001F1E0FFEF6003026CE3900006E0FFD4
:106C4700EF70037F0122305C05127785800312778E
:106C57008B204A037F0022128CD3EF6401707A30B5
:106C67004A74C24A900052E0FF9001EDEFF09000A5
:106C770053E0FF9001EEEFF0900051E0FF9001EF3D
:106C8700EFF09001EFE0FFEFB41F199001EBE0FF89
:106C97009001EEE0FEEEB5070B12778B900006E44D
:106CA700F07F01229001EAE0FF9001EDE0FEEEB5F2
:106CB700070E9001EBE0FF9001EEE0FEEE6F60093A
:106CC7009001F17401F07F0022900096E0FF9000A0
:106CD70006EFF07F00227F00227F00229001F1E083
:106CE700FFEF64016003026D8A900006E0FFEF701A
:106CF700037F0122305C05127785800312778B2092
:106D07005C089001F1E4F07F0122204A037F002212
:106D1700C24A900052E0FF9001EDEFF0900053E07F
:106D2700FF9001EEEFF0900051E0FF9001EFEFF0E0
:106D37009001EFE0FFEFB41F199001EBE0FF900126
:106D4700EEE0FEEEB5070B12778B900006E4F07FBE
:106D570001229001EAE0FF9001EDE0FEEEB5072089
:106D67009001EBE0FF9001EEE0FEEEB50712900018
:106D770096E0FF900006EFF09001F1E4F07F00222B
:0B6D87007F00229001F1E4F07F002269
:108CD30090008DE0FFEF600D1277AF40047F0180BD
:108CE300027F00222290008EE0FFEF601390008F3E
:108CF300E0FFE534D39F40047F0122227F0022223C
:108D030090008FE0FFE534C39F50047F0122227F50
:028D130000223C
:106507009001F8E0FFEF60030265C7900008E0FF25
:10651700EF70037F0122205C0B12778B900008E459
:10652700F07F0122128CD3EFB40105127785800327
:1065370012778B9001F7E0FFEFB40106203B037F52
:1065470000229001F7E0FFEFB402062041037F002D
:1065570022128CD3EF640170649001F7E0FFEF64BF
:10656700017021303B1EC23BE54165406009900147
:10657700F87401F07F002290009BE0FF900008EF85
:10658700F07F00229001F7E0FFEF6402702F3041A7
:106597002CC2419001FAE536F09001FAE0FF900134
:1065A700F9E0FEEE6F60099001F87401F07F0022B8
:1065B70090009BE0FF900008EFF07F00227F002211
:1065C7009001F8E0FFEF6401600302668490000821
:1065D700E0FFEF70037F0122205C1012778B9001A0
:1065E700F8E4F0900008E4F07F0122128CD3EFB4B6
:1065F7000105127785800312778B9001F7E0FFEF93
:10660700B40106203B037F00229001F7E0FFEFB4BF
:1066170002062041037F0022128CD3EF6401705AD7
:106627009001F7E0FFEFB4011C303B19C23BE54195
:10663700B540129001F8E4F090009BE0FF9000084D
:10664700EFF07F00229001F7E0FFEF6402702B303C
:106657004128C2419001FAE536F09001FAE0FF9037
:1066670001F9E0FEEEB507129001F8E4F090009B07
:10667700E0FF900008EFF07F00227F00229001F8F2
:05668700E4F07F002299
:1087BD007BFF7A887924128F621277AF400B7BFF93
:1087CD007A887935128F9780097BFF7A88794612DE
:1087DD008F977F17127961AF3412784690005EE063
:1087ED00FF12793290005FE0FF127932900060E065
:1087FD00FF1279327F1C127961AF331278469000E7
:10880D005EE0FF12793290005FE0FF127932900046
:07881D0060E0FF1279322236
:10905700900092E0FFEF6013900093E0FFE533D3B9
:109067009F40047F0122227F002222900093E0FF8D
:0D907700E533C39F50047F0122227F0022B9
:1092C80090008DE0FFEF60071284761286722212FA
:0692D8006971126EE9222B
:10847600900201E0FFEF70161277AF407290009005
:10848600E0FF90000AEFF0900201E004F022900273
:1084960001E0FFEF640170281277AF401C90000ADC
:1084A600E0FFEF704AD25C90009AE0FF90000CEF7C
:1084B600F0900201E004F02222900201E4F0222270
:1084C600900201E0FFEFB402211277AF400B90005B
:1084D6009AE0FF90000CEFF02290000CE0FFEF70A6
:1084E6000EC25C900201E4F02222900201E4F02226
:10697100900201E0FFEF704C90008EE0FFEF60238A
:1069810090008FE0FFE534D39F4013900090E0FF2B
:1069910090000AEFF0900201E004F0228026C25C30
:1069A10022802190008FE0FFE534C39F50139000B7
:1069B10090E0FF90000AEFF09002017403F0228052
:1069C10003C25C22900201E0FFEF64017035900088
:1069D1008FE0FFEF24FBFFE534D39F401F90000AB7
:1069E100E0FFEF6003026AD4D25C900091E0FF9077
:1069F100000CEFF0900201E004F02222900201E489
:106A0100F02222900201E0FFEF6402702E90008FCD
:106A1100E0FFEF24FBFFE534D39F400B900091E0B2
:106A2100FF90000CEFF02290000CE0FFEF600302FA
:106A31006AD4C25C900201E4F02222900201E0FFDC
:106A4100EF6403704390008FE0FF7E00EF2405FFA9
:106A5100EE3400FEAD347C00C3ED9FEE6480F8ECB3
:106A6100648098501C90000AE0FFEF7066D25C9041
:106A71000091E0FF90000CEFF0900201E004F022A1
:106A810022900201E4F02222900201E0FFEF64046F
:106A9100703C90008FE0FF7E00EF2405FFEE340094
:106AA100FEAD347C00C3ED9FEE6480F8EC64809809
:106AB100500B900091E0FF90000CEFF02290000C41
:106AC100E0FFEF700EC25C900201E4F0222290021E
:046AD10001E4F022CA
:106EE900900202E0FFEF704C90008EE0FFEF60230C
:106EF90090008FE0FFE534D39F4013900090E0FFAE
:106F090090000BEFF0900202E004F0228026C25DAF
:106F190022802190008FE0FFE534C39F5013900039
:106F290090E0FF90000BEFF09002027403F02280D2
:106F390003C25D22900202E0FFEF6401703190000C
:106F49008FE0FFEF24FBFFE534D39F401B90000B3C
:106F5900E0FFEF600302703BD25D90000D7464F0B6
:106F6900900202E004F02222900202E4F022229030
:106F79000202E0FFEFB4022A90008FE0FFEF24FB4A
:106F8900FFE534D39F400790000D740AF02290006A
:106F99000DE0FFEF600302703BC25D900202E4F076
:106FA9002222900202E0FFEF6403703F90008FE01D
:106FB900FF7E00EF2405FFEE3400FEAD347C00C3F4
:106FC900ED9FEE6480F8EC648098501890000BE017
:106FD900FFEF705ED25D90000D7464F0900202E0E4
:106FE90004F02222900202E4F02222900202E0FF41
:106FF900EF6404703890008FE0FF7E00EF2405FFF6
:10700900EE3400FEAD347C00C3ED9FEE6480F8ECF5
:10701900648098500790000D7464F02290000DE090
:10702900FFEF700EC25D900202E4F022229002028C
:03703900E4F0225E
:10867200900202E0FFEF70161277AF406A9000900E
:10868200E0FF90000BEFF0900202E004F022900273
:1086920002E0FFEF640170241277AF401890000BE4
:1086A200E0FFEF7042D25D90000D7464F090020220
:1086B200E004F02222900202E4F02222900202E080
:1086C200FFEFB4021D1277AF400790000D7464F003
:1086D2002290000DE0FFEF700EC25D900202E4F006
:0886E2002222900202E4F022C2
:109282001283F58F7D900249E0FFEF657D600890C3
:079292000249E57DF0D25E08
:0192990022B2
:1081E1007BFF7A887957128F97900207E0FFEF752E
:1081F100F06484FFEF2430F571900207E0FFEF7522
:10820100F06484AFF0EF75F00A84FFEF2430F5726B
:10821100900207E0FFEF75F06484AFF0EF75F00AAC
:1082210084AFF0EF2430F5737F16127961AF7112CC
:108231007932AF72127932AF731279327F1F1279AC
:1082410061900065E0FFEF75F00A84FFEF2430F5DF
:1082510071900065E0FFEF75F00A84AFF0EF243014
:0C826100F572AF71127932AF72127932EF
:01826D0022EE
:10917E00900204E0FFEF701D7BFF7A887968128FF2
:10918E0062900003740AF0900003E0FFEF70F87530
:06919E00840075EF0322BE
:10615400757600757509D3E5756480948640677516
:106164007413C3E574648094804057AF74EF33951F
:10617400E0FE74C92FF58274003EF583E0FFEF65FD
:1061840075703BE57404FFAE76EE25E024F1F582EC
:10619400E43400F583EFF0AF76EF25E024F2F582E6
:1061A400E43400F583E575F00576E576D394144080
:1061B4000D7BFF7A887979128F62D25F800415741F
:1061C40080A015758090757506D3E57564809480FC
:1061D4004067757400C3E574648094945057AF7439
:1061E400EF3395E0FE74C92FF58274003EF583E029
:1061F400FFEF6575703BE57404FFAE76EE25E02491
:10620400F1F582E43400F583EFF0AF76EF25E02476
:10621400F2F582E43400F583E575F00576E576D38E
:106224009414400D7BFF7A887979128F62D25F8053
:1062340004057480A015758090E5766414600B7B6A
:10624400FF7A887979128F62D25F75760075750945
:10625400D3E575648094864067757400C3E57464FF
:106264008094945057AF74EF3395E0FE74C92FF5C2
:106274008274003EF583E0FFEF6575703BE57404BE
:10628400FFAE76EE25E02419F582E43401F583EFC0
:10629400F0AF76EF25E0241AF582E43401F583E5C6
:1062A40075F00576E576D39414400D7BFF7A8879F2
:1062B40079128F62D25F8004057480A01575809076
:1062C400757506D3E575648094804067757413C34F
:1062D400E574648094804057AF74EF3395E0FE74A6
:1062E400C92FF58274003EF583E0FFEF6575703BBE
:1062F400E57404FFAE76EE25E02419F582E434015A
:10630400F583EFF0AF76EF25E0241AF582E434014B
:10631400F583E575F00576E576D39414400D7BFF9F
:106324007A887979128F62D25F8004157480A015FF
:10633400758090E5766414600B7BFF7A8879791216
:046344008F62D25F33
:016348002232
:1049CA002020464C45584956203030392020202096
:1049DA0000527074724E756D62657257726F6E67AF
:1049EA00210050726F6772616D6D696E67526573EF
:1049FA006574002049502050524F4752414D4D494D
:104A0A004E47200043544353532036332E30202040
:104A1A002020202043544353532036372E30202061
:104A2A002020202043544353532036392E3420204B
:104A3A002020202043544353532037312E3920203D
:104A4A002020202043544353532037342E3420202F
:104A5A002020202043544353532037372E30202020
:104A6A002020202043544353532037392E37202007
:104A7A002020202043544353532038322E352020FF
:104A8A002020202043544353532038352E342020ED
:104A9A002020202043544353532038382E352020D9
:104AAA002020202043544353532039312E352020CF
:104ABA002020202043544353532039342E382020B9
:104ACA002020202043544353532039372E342020AA
:104ADA00202020204354435353203130302E30209D
:104AEA00202020204354435353203130332E352085
:104AFA00202020204354435353203130372E322074
:104B0A00202020204354435353203131302E392062
:104B1A00202020204354435353203131342E38204F
:104B2A00202020204354435353203131382E38203B
:104B3A00202020204354435353203132332E302037
:104B4A00202020204354435353203132372E332020
:104B5A00202020204354435353203133312E382010
:104B6A00202020204354435353203133362E3520FE
:104B7A00202020204354435353203134312E3320F4
:104B8A00202020204354435353203134362E3220E0
:104B9A00202020204354435353203135312E3420D2
:104BAA00202020204354435353203135362E3720BA
:104BBA00202020204354435353203135392E3820A6
:104BCA00202020204354435353203136322E3220A2
:104BDA00202020204354435353203136352E35208C
:104BEA00202020204354435353203136372E392076
:104BFA00202020204354435353203137312E332071
:104C0A00202020204354435353203137332E382059
:104C1A00202020204354435353203137372E33204A
:104C2A00202020204354435353203137392E392032
:104C3A00202020204354435353203138332E35202B
:104C4A00202020204354435353203138362E32201B
:104C5A00202020204354435353203138392E392001
:104C6A00202020204354435353203139322E3820F8
:104C7A00202020204354435353203139362E3620E6
:104C8A00202020204354435353203139392E3520D4
:104C9A00202020204354435353203230332E3520D2
:104CAA00202020204354435353203230362E3520BF
:104CBA00202020204354435353203231302E3720B2
:104CCA00202020204354435353203231382E3120A0
:104CDA00202020204354435353203232352E37208C
:104CEA00202020204354435353203232392E31207E
:104CFA00202020204354435353203233332E36206E
:104D0A00202020204354435353203234312E38205C
:104D1A00202020204354435353203235302E332051
:104D2A00202020204354435353203235342E31203F
:104D3A002020202020202020202020202020202069
:044D4A0020202020E5
:105F590075840F12634912935B7BFF7A4979CA12E0
:105F69008F6212778520A10875840F43E8C08006E7
:105F790075840F53E83F1292DE9000037401F0908C
:105F89000003E070FA90024D7401F090024E740320
:105F9900F07D007CFC7F10128DD1E490024DF090D1
:105FA900024EF0C25F1290DD900065E0FF6005D3FC
:105FB900941440119000657401F07BFF7A4979DBF4
:105FC900128F62D25F205F121281E1127EFD128967
:105FD900B8128A14129029126154900204740FF0B5
:105FE90012777912779D9000A3E0FF90000EE4F0FC
:105FF900A3EFF09000AEE0900203F0E4900147F0C7
:106009009001E9F09001E8F09001F1F09001FBF0C6
:1060190090005C74FFF090005DF0E4900249F0900C
:106029000248F0F50AC264C261C2629001F0F0123E
:10603900778B900243740FF0304313123E9F1290F6
:10604900DD127EFD1289B8128A14C24380EA20A6A5
:106059000E1287BDE49001E9F09001E8F080EF307D
:10606900461DC246123E9F1290DD127EFD1289B86E
:10607900128A1412935BE49001E8F09001E9F0436D
:10608900E740305806128955129132125444123A97
:106099006212680A90024AE0B4551F90024BE0B4BC
:1060A900AA1890024C7414F090024CE070FA7BFF2D
:1060B9007A4979EC128F6212777F127791503B12ED
:1060C900917E12703C1275271258871292C812924B
:1060D90082305E1E20611BC25E900249E02400FEF0
:1060E900E43417900223F0A3CEF090021F7401F05C
:1060F900D261E4900252F00260571277799000BEA3
:10610900E0600312779D9000A3E0FF90000EE4F099
:10611900A3EFF09000AEE0900203F0E49001E9F003
:106129009001E8F09001F1F0900065E090005CF0DA
:1061390090005D74FCF012778B900204741EF07B62
:0B614900FF7A4979FD12668C02605756
:10888A0001AE01C901DA01EB01FC020E022002333A
:10889A000247025C02710287029902AB02C302DC40
:1088AA0002F50310032B03480365038403A403C5DD
:1088BA0003E6040A042E04430453046A047A049166
:1088CA0004A204BA04CC04E504F705100524053E05
:1088DA000552056D0582059E05D10605061C063B57
:0688EA00067306AD06C78F
:10924800C23DC23FEF25E0248AF582E43488F583E5
:0E925800E493F51A740193F51BD23ED238222E
:0F934C00C23DC23EC238C23FE4787EF6C257220D
:0300A300028C903C
:108C9000C0E0C0F0C083C082C0D075D000C000C0AA
:108CA00001C002C003C004C005C006C007205805AB
:108CB000127A9680031288F0D007D006D005D0042F
:108CC000D003D002D001D000D0D0D082D083D0F059
:038CD000D0E032BF
:030093000286EAF8
:0B86EA00C0E0C0D075D000C006C00783
:1086F500AE84758402E5357007AFBE75BB07802F64
:10870500E535B40107AFBE75BB048023E535B4027A
:1087150007AFBE75BB068017E535B4030885BE33C4
:1087250075BB04800AE535B40409AFBE75BB050504
:10873500358010E535B4050885BE3475BB04800069
:07874500753500C2ED8E84C2
:09874C00D007D006D0D0D0E032F5
:03008300028D9457
:108D9400C0E0C0F0C083C082C0D075D000C000C0A5
:108DA40001C002C003C004C005C006C007C2CF1280
:108DB4001FCAD007D006D005D004D003D002D001FA
:0D8DC400D000D0D0D082D083D0F0D0E032EB
:03007300028151B6
:10815100C0E0C0F0C083C082C0D075D000C000C0F4
:1081610001C002C003C004C005C006C007C2CF30B1
:1081710058051287558003128AC97898E66001165E
:10818100304027C240D54C05754C0A054B1272BAD6
:10819100D51C09751C0A758401438820D5301B75CF
:1081A10030607584024388208010D24012749D781B
:1081B1009916E670057604121BF875840143881040
:1081C100758402D2ECD007D006D005D004D003D0FC
:1081D10002D001D000D0D0D082D083D0F0D0E03214
:03006B00028BBF46
:108BBF00C0E0C0F0C083C082C0D075D000C000C07C
:0D8BCF0001C002C003C004C005C006C007FD
:0E8BDC0085846D127655758402C28D856D8478
:108BEA00D007D006D005D004D003D002D001D000DF
:0B8BFA00D0D0D082D083D0F0D0E03289
:03005B00028B71A4
:108B7100C0E0C0F0C083C082C0D075D000C000C0CA
:108B810001C002C003C004C005C006C0071257BC23
:108B9100789AE6600116900007E0600214F075848F
:108BA10001C28DD007D006D005D004D003D002D0A9
:0E8BB10001D000D0D0D082D083D0F0D0E032FE
:03005300028C0517
:108C0500C0E0C0F0C083C082C0D075D000C000C035
:108C150001C002C003C004C005C006C007C28C3035
:108C25005A04C25A8005D25A1272DCD007D006D037
:108C350005D004D003D002D001D000D0D0D082D04E
:068C450083D0F0D0E03204
:0300230002931A2B
:10931A00309904C299C266309807859908C298D2D2
:02932A006532AA
:108C4B00A984A2AF9267AEB1C2AF75840F53A1FED8
:108C5B008FB1E4F58490024DE042B790024EE042B2
:108C6B008F8C658D668D828C83EBF0E4F58490029E
:108C7B004EE0F4528F90024DE0F452B78EB18984DE
:048C8B00A26792AF9B
:018C8F0022C2
:108DD100A984A2AF9267AEB1C2AF8C658D668FB127
:108DE100E4F58490024DE0FF42B7E4F58490024E31
:108DF100E0FD428F856682856583E4F0EDF4528F54
:0C8E0100EFF452B78EB18984A26792AFE3
:018E0D002242
:1091E900AE84A2AF9267ABB1C2AF8FB18C678D6805
:0F91F9008D828C83E493FF8BB18E84A26792AF3B
:019208002243
:100EC800506172616D657465727357726F6E6721D8
:100ED800002020464C4558495620303039202020E3
:100EE80020002020202020202020202020204944CD
:100EF8004C45004E4F204C54522042555320204917
:100F0800444C452000204D757469706C65204D6116
:100F1800737465727320002054657374696E67205A
:100F28004D6F64652020200043726F7373204275F3
:100F3800737920434F5320200043726F737320420C
:100F48007573792053454E53450053656E642049A7
:100F5800646C654D657373616765002020474F5465
:100F68004F204D45535341474520200020205365CD
:100F78006E64696E67204357494420200020435718
:100F88004944205544544420464C4147200044538A
:100F9800502046494E49534853204357494400314D
:100FA8003357414954205544544420464C41470046
:100FB800323157414954205544544420464C414706
:100FC80000333357414954205544544420464C413A
:100FD8004700333757414954205544544420464C20
:100FE8004147004C5452564F4950204F5554474F93
:100FF800494E4700343457414954205544544420FD
:10100800464C4147003438574149542055445444CC
:1010180020464C41470035305741495420554454E7
:101028004420464C414700204C6F63616C20486166
:101038006E672054696D6500353357414954205512
:1010480044544420464C4147005761697420436129
:10105800727269657244726F70003537574149542E
:10106800205544544420464C41470020564F49508F
:10107800204F5554474F494E4720200020564F498E
:10108800502048616E672054696D652000205761C3
:1010980069744E6574776F726B48616E6700363499
:1010A80057414954205544544420464C4147003642
:1010B8003857414954205544544420464C41470030
:1010C800373057414954205544544420464C4147F1
:1010D800002020494E434F4D494E47204C54522042
:1010E8002000373357414954205544544420464C36
:1010F8004147003738574149542055445444204605
:101108004C414700383057414954205544544420F5
:10111800464C4147002020494E434F4D494E4720F9
:1011280043544353532020002020494E434F4D49F8
:101138004E47204443532020003834574149542017
:101148005544544420464C41470038385741495487
:10115800205544544420464C41470043726F7373F2
:101168002042757379204D6F6465310043726F7347
:10117800732042757379204D6F6465320043726F36
:1011880073732042757379204D6F64653300437221
:101198006F73732042757379204D6F64653400391D
:1011A8003357414954205544544420464C41470044
:1011B80043544353532036332E3020202020202000
:1011C80043544353532036372E30202020202020EC
:1011D80043544353532036392E34202020202020D6
:1011E80043544353532037312E39202020202020C8
:1011F80043544353532037342E34202020202020BA
:1012080043544353532037372E30202020202020AA
:1012180043544353532037392E3720202020202091
:1012280043544353532038322E3520202020202089
:1012380043544353532038352E3420202020202077
:1012480043544353532038382E3520202020202063
:1012580043544353532039312E3520202020202059
:1012680043544353532039342E3820202020202043
:1012780043544353532039372E3420202020202034
:101288004354435353203130302E30202020202027
:101298004354435353203130332E3520202020200F
:1012A8004354435353203130372E322020202020FE
:1012B8004354435353203131302E392020202020ED
:1012C8004354435353203131342E382020202020DA
:1012D8004354435353203131382E382020202020C6
:1012E8004354435353203132332E302020202020C2
:1012F8004354435353203132372E332020202020AB
:101308004354435353203133312E3820202020209A
:101318004354435353203133362E35202020202088
:101328004354435353203134312E3320202020207E
:101338004354435353203134362E3220202020206A
:101348004354435353203135312E3420202020205C
:101358004354435353203135362E37202020202044
:101368004354435353203135392E38202020202030
:101378004354435353203136322E3220202020202C
:101388004354435353203136352E35202020202016
:101398004354435353203136372E39202020202000
:1013A8004354435353203137312E332020202020FB
:1013B8004354435353203137332E382020202020E4
:1013C8004354435353203137372E332020202020D5
:1013D8004354435353203137392E392020202020BD
:1013E8004354435353203138332E352020202020B6
:1013F8004354435353203138362E322020202020A6
:101408004354435353203138392E3920202020208B
:101418004354435353203139322E38202020202082
:101428004354435353203139362E36202020202070
:101438004354435353203139392E3520202020205E
:101448004354435353203230332E3520202020205C
:101458004354435353203230362E35202020202049
:101468004354435353203231302E3720202020203C
:101478004354435353203231382E3120202020202A
:101488004354435353203232352E37202020202016
:101498004354435353203232392E31202020202008
:1014A8004354435353203233332E362020202020F8
:1014B8004354435353203234312E382020202020E7
:1014C8004354435353203235302E332020202020DC
:1014D8004354435353203235342E312020202020CA
:1014E80020202020202020202020202020202020F4
:1014F8004443532030303620494E56203032312074
:101508004443532030303720494E5620323134205E
:101518004443532030313520494E56203134312050
:101528004443532030313720494E5620303530203F
:101538004443532030323120494E56203030362033
:101548004443532030323320494E5620303437201C
:101558004443532030323520494E5620323434200B
:101568004443532030323620494E562034363420F6
:101578004443532030333120494E562036323720E9
:101588004443532030333220494E562030353120E1
:101598004443532030333620494E562031373220C9
:1015A8004443532030343320494E562034343520B8
:1015B8004443532030343720494E562030323320AC
:1015C8004443532030353020494E5620303137209F
:1015D8004443532030353120494E56203033322091
:1015E8004443532030353320494E56203435322079
:1015F8004443532030353420494E5620343133206B
:101608004443532030363520494E56203237312056
:101618004443532030373120494E5620333036204A
:101628004443532030373220494E56203234352037
:101638004443532030373320494E56203530362026
:101648004443532030373420494E56203137342014
:101658004443532031313420494E5620373132200B
:101668004443532031313520494E562031353220FC
:101678004443532031313620494E562037353420E3
:101688004443532031323220494E562032323520DD
:101698004443532031323520494E562033363520C5
:1016A8004443532031333120494E562033363420B9
:1016B8004443532031333220494E562035343620A6
:1016C8004443532031333420494E5620323233209C
:1016D8004443532031343120494E5620303135208F
:1016E8004443532031343320494E5620343132207C
:1016F8004443532031343520494E56203237342064
:101708004443532031353220494E5620313135205B
:101718004443532031353520494E56203733312044
:101728004443532031353620494E56203236352031
:101738004443532031363220494E56203530332029
:101748004443532031363520494E56203235312016
:101758004443532031373220494E56203033362007
:101768004443532031373420494E562030373420F3
:101778004443532032303520494E562032363320E8
:101788004443532032313220494E562033353620D7
:101798004443532032313420494E562030303720CC
:1017A8004443532032323320494E562031333420BB
:1017B8004443532032323520494E562031323220AC
:1017C8004443532032323620494E5620343131209A
:1017D8004443532032343320494E56203335312088
:1017E8004443532032343420494E56203032352079
:1017F8004443532032343520494E56203037322066
:101808004443532032343620494E56203532332053
:101818004443532032353120494E56203136352045
:101828004443532032353220494E56203436322034
:101838004443532032353520494E5620343436201F
:101848004443532032363120494E56203733322014
:101858004443532032363320494E56203230352007
:101868004443532032363520494E562031353620F0
:101878004443532032363620494E562034353420DE
:101888004443532032373120494E562030363520D4
:101898004443532032373420494E562031343520C2
:1018A8004443532033303620494E562030373120B8
:1018B8004443532033313120494E562036363420A4
:1018C8004443532033313520494E56203432332097
:1018D8004443532033323520494E56203532362082
:1018E8004443532033333120494E56203436352073
:1018F8004443532033333220494E56203435352063
:101908004443532033343320494E56203533322054
:101918004443532033343620494E56203631322042
:101928004443532033353120494E56203234332036
:101938004443532033353620494E56203231322025
:101948004443532033363420494E56203133312016
:101958004443532033363520494E56203132352002
:101968004443532033373120494E562037333420EF
:101978004443532034313120494E562032323620E8
:101988004443532034313220494E562031343320D9
:101998004443532034313320494E562030353420C7
:1019A8004443532034323320494E562033313520B6
:1019B8004443532034333120494E562037323320A4
:1019C8004443532034333220494E56203531362093
:1019D8004443532034343520494E56203034332084
:1019E8004443532034343620494E5620323535206E
:1019F8004443532034353220494E56203035332065
:101A08004443532034353420494E5620323636204C
:101A18004443532034353520494E56203333322041
:101A28004443532034363220494E56203235322032
:101A38004443532034363420494E56203032362021
:101A48004443532034363520494E56203333312011
:101A58004443532034363620494E562036363220F9
:101A68004443532035303320494E562031363220F6
:101A78004443532035303620494E562030373320E2
:101A88004443532035313620494E562034333220D2
:101A98004443532035323320494E562032343620C1
:101AA8004443532035323620494E562033323520B0
:101AB8004443532035333220494E562033343320A3
:101AC8004443532035343620494E56203133322092
:101AD8004443532035363520494E5620373033207D
:101AE8004443532036303620494E56203633312071
:101AF8004443532036313220494E56203334362061
:101B08004443532036323420494E5620363332204F
:101B18004443532036323720494E56203033312043
:101B28004443532036333120494E56203630362030
:101B38004443532036333220494E5620363234201F
:101B48004443532036353420494E56203734332009
:101B58004443532036363220494E562034363620F8
:101B68004443532036363420494E562033313120F1
:101B78004443532037303320494E562035363520DC
:101B88004443532037313220494E562031313420D6
:101B98004443532037323320494E562034333120C2
:101BA8004443532037333120494E562031353520B0
:101BB8004443532037333220494E562032363120A1
:101BC8004443532037333420494E5620333731208D
:101BD8004443532037343320494E56203635342079
:101BE8004443532037353420494E5620313136206E
:10703C00305F097BFF7A0E79C8028F629000BDE049
:10704C00FFB4010E90005C74FFF0E490005DF00260
:10705C007174EF640260030271271277739000BEA3
:10706C00E06003127797787EE66003027116305762
:10707C00030271169001F0E07032D23F9000A4E050
:10708C0024FF924E900065E0FF9001B4F09000A2B6
:10709C00E09001B5F09001B6EFF01283749001B757
:1070AC00EFF0127E629001F07402F022127B77EF07
:1070BC0064017050D23F9001B4E024DCF582E434DA
:1070CC0000F583E024FF924E9001B2E0FF249CF582
:1070DC0082E43401F583E09001B4F074872FF582DB
:1070EC00E43401F583E09001B5F09001B2E0900139
:1070FC00B6F012826E9001B7EFF0127E629001F042
:10710C00E014F0229001F0E014F0900065E09000A3
:10711C005CF09000A2E090005DF0229001E8E0B4F9
:10712C000A005043907137F8282873027155027188
:10713C005802715B02715E027161027164027167C7
:10714C0002716A02716D0271700228CF027DB70262
:10715C0080C00242B00230CE024D4E0250CA0235FF
:10716C00C402463F025AD7E49001E8F09001E9F0DE
:01717C0022F0
:1028CF009001E9E0B40B0040030230229028E2F8B7
:1028DF00282873022903022947022BFD022C3D02EF
:1028EF002C5C022C7E022D49022DD3022E69022E62
:1028FF0087022F73E4900248F0900245F0C2397BB3
:10290F00FF7A0E79D9128F627BFF7A0E79EA128FD6
:10291F0097E4900251F090005C74FFF090005DF02E
:10292F001277799000BEE0600312779D12934C905E
:10293F0001E97401F0023027900243E06020900219
:10294F0044E0701A900251E06014E4F07BFF7A0EBD
:10295F0079D9128F627BFF7A0E79EA128F979002E4
:10296F0043E07014900251E06401600C7401F07B3D
:10297F00FF7A0E79FB128F97900244E06017900256
:10298F0051E06402600F7402F07BFF7A0F790D1231
:10299F008F9702302720A55F1277739000BEE060FB
:1029AF00031277979000BBE0900000F0900065E075
:1029BF00FF90005CF09000A2E0FE90005DF09001AF
:1029CF00E97405F09001B4EFF09001B5EEF09000CE
:1029DF0065E09001B6F012826E9001B7EFF09000B3
:1029EF00A4E024FF924E127E62D23F7BFF7A0F79D2
:1029FF001F128F62023027305C60304A5DC24A90EE
:102A0F000052E0FFC39415505174DC2FF582E4346B
:102A1F0000F583E0FFA248E4336F703EA24892496D
:102A2F00900052E09001EAF0900053E09001EBF03B
:102A3F00900051E09001ECF0126D929001ECE06487
:102A4F001F60179001EAE0FF9001EBE0FD7C0012A0
:102A5F007F989001E87402022E83C24A1291A4BF9C
:102A6F0001211277739000BEE060031277979000F8
:102A7F005C74FFF090005DF09000BBE0900000F000
:102A8F00022E4F9000BFE0FF64016004EFB4020B11
:102A9F00305C087BFF7A0F793080199000BFE0FF20
:102AAF0064036004EFB4041F129057BF01197BFF3A
:102ABF007A0F7941128F6290009CE078A1F6900115
:102ACF00E97409F0023027128CD3EF64017065307E
:102ADF003B28C23B9001F704F0D239854041E541D4
:102AEF0075F010A424B8F9741135F0FA7BFF128F2A
:102AFF0062AF411285F5C239802A304137C2419009
:102B0F0001F9E536F075F010A424F8F9741435F0D6
:102B1F00FA7BFF128F629001F9E0FF1282F19001B0
:102B2F00F77402F09001E9740AF090009CE078A12C
:102B3F00F6023027C23BC24190000EE07002A3E0C4
:102B4F0070409000A3E0603A7BFF7A0F7952128FAA
:102B5F00629000A3E0FF90000EE4F0A3EFF090006E
:102B6F005C74FFF090005DF01277739000BEE06030
:102B7F00031277979000BBE0900000F09001E902FC
:102B8F002FD6900206E060030230279000AEE0FFE0
:102B9F007003023027900203E06003023027900099
:102BAF00ACE0FE601070030230279001FDE064017D
:102BBF006003023027900203EFF0E49001FDF01262
:102BCF0077739000BEE060031277979000BBE090A0
:102BDF000000F0900065E090005CF090005D74FDE7
:102BEF00F0E49001E9F09001E804F0023027900042
:102BFF0000E0600302302730570302302790006552
:102C0F00E0FF9001B4F09001B574FFF09001B6EFC2
:102C1F00F09001B7F09000A4E024FF924E127E6274
:102C2F00D23F126E349001E97403F0023027787EA0
:102C3F00E66003023027305703023027900097E0F9
:102C4F00900001F09001E97404F002302790000128
:102C5F00E060030230271277799000BEE060031224
:102C6F00779DE49001E9F09001FD04F002302730E8
:102C7F00A503022FDB900065E090005CF09000A2AE
:102C8F00E090005DF0128CD3BF01051277858003B1
:102C9F0012778B787EE660030230273057030230BD
:102CAF00279001F0E07037D23F9000A4E024FF920C
:102CBF004E900065E0FF9001B4F09000A2E090010B
:102CCF00B5F09001B6EFF01283749001B7EFF012E8
:102CDF007E629001F07402F0126E34023027127B84
:102CEF0077EF6401704BD23F9001B2E0FF249CF567
:102CFF0082E43401F583E09001B4F074872FF582FC
:102D0F00E43401F583E09001B5F09001B2E0900159
:102D1F00B6F012826E9001B7EFF09001B4E024DCB0
:102D2F00F582E43400F583E024FF924E127E628038
:102D3F00009001F0E014F0023027900000E06003F3
:102D4F00023027305703023027787EE660030230C7
:102D5F002790005C74FFF090005DF0127C45EF64EB
:102D6F00016003022E589001B2E0FF249CF582E42B
:102D7F003401F583E09001B4F074872FF582E434C9
:102D8F0001F583E09001B5F09001B2E09001B6F04B
:102D9F0012001C9001B7EFF09001B4E024DCF58233
:102DAF00E43400F583E024FF924E127E62D23F7B23
:102DBF00FF7A0F7963128F62126E349001E97407F4
:102DCF00F0023027305C63304A62C24A900052E012
:102DDF00FFC39415505674DC2FF582E43400F5834D
:102DEF00E0FFA248E4336F7043A24892499000522B
:102DFF00E09001EAF0900053E09001EBF090005169
:102E0F00E09001ECF0126D929001ECE0641F601CF9
:102E1F009001EAE0FF9001EBE0FD7C00127F98E467
:102E2F009001E9F09001E8022FD6C24A787EE66061
:102E3F00030230273057030230271291A4EF6009A5
:102E4F009001E97406F0023027900097E09000019E
:102E5F00F09001E97408F0023027900001E0600360
:102E6F000230271277799000BEE0600312779D90B1
:102E7F0001FD7401F0023022305C63304A60C24AB7
:102E8F00900052E0FFC39415505474DC2FF582E488
:102E9F003400F583E0FFA248E4336F7041A24892FB
:102EAF0049900052E09001EAF0900053E09001EB5E
:102EBF00F0900051E09001ECF0126D929001ECE077
:102ECF00641F601A9001EAE0FF9001EBE0FD7C00C7
:102EDF00127F98E49001E9F09001E8022FD6C24AE0
:102EEF009000BFE0FF64016004EFB4020A205C07AA
:102EFF009001E97401F022EF64036004EFB4040C55
:102F0F00129057EF70069001E904F02278A1E66065
:102F1F0003023027900065E090005CF090005D7434
:102F2F00FDF09000BFE0FF64016004EFB4020530D4
:102F3F005C02801C9000BFE0FF64036008EF640434
:102F4F006003023027129057EF64016003023027AD
:102F5F0090009DE0900005F0E49001E9F09001E809
:102F6F007409F022128CD3EF64017060304A5FC293
:102F7F004A900052E0FFC39415505374DC2FF58232
:102F8F00E43400F583E0FFA248E4336F7040A248B9
:102F9F009249900052E09001EAF0900053E09001C6
:102FAF00EBF0900051E09001ECF0126D929001EC7B
:102FBF00E0641F60199001EAE0FF9001EBE0FD7CF7
:102FCF0000127F989001E87402F0804C8045C24A4D
:102FDF0078A1E67043305C40900068E07004C2391D
:102FEF0080321277739000BEE060031277971277EA
:102FFF00859000BBE0900000F0900065E090005CD1
:10300F00F090005D74FEF0E49001E9F09001E87437
:10301F0005F022E49001E9F0900245E0640370416D
:10302F001277739000BEE060031277979000BBE0B9
:10303F00900000F0E4900245F0900246E0FF90000F
:10304F005CF0900247E0FE90005DF09001EAEFF037
:10305F009001EBEEF0E49001E9F09001E87407F0D5
:10306F0022900245E060571277739000BEE0600334
:10307F001277979000BBE0900000F0900065E09011
:10308F00005CF090005D74FEF0900245E0FFB4012B
:10309F000C9001F77401F0900247E0F541EFB40294
:1030AF000E9001F77402F0900247E09001F9F0E4FE
:0F30BF00900245F09001E9F09001E87408F022CA
:107DB700128A709001E9E0702C20612190022374EF
:107DC70018F0A37402F090021F14F0D2619001E939
:107DD700F07BFF7A0F7974128F6202798A7BFF7AC0
:107DE7000F798580699001E9E0B40120900248E0AD
:107DF70064017066F0900097E0900001F09001E94F
:107E07007402F07BFF7A0F7996028F629001E9E0A6
:107E1700B40219900001E070411277799000BEE03A
:107E2700600312779D9001E97403F0229001E9E065
:107E3700B4031E2061129002237418F0A3E4F0909B
:107E4700021F04F0D26180097BFF7A0F79A7028FA6
:0B7E570097E49001E8F09001E9F022B0
:1080C0009001E9E0703B900072E0602B12777390B2
:1080D00000BEE060031277979000BBE0900000F0D4
:1080E0009001EAE090005CF09001EBE090005DF020
:1080F0009001E97401F022E49001E9F09001E8F0C8
:10810000229001E9E06401703E2061329001EAE0D2
:10811000FE9001EBE07C002400FFEC3E900223F097
:10812000A3EFF090021F7401F0D261900073E09011
:1081300001E86004740480027403F0E4800E7BFFA5
:108140007A0F79B8028F97E49001E8F09001E9F096
:01815000220C
:1042B0009001E9E0704A900000E0600302463EA2EF
:1042C00049924E9001EAE09001B4F09001EBE09049
:1042D00001B5F0900065E09001B6F0128374900192
:1042E000B7EFF0127E62D23F126E349001F0740884
:1042F000F0900096E0900006F09001E97401F02241
:104300009001E9E06401703E126C37EF6002805565
:10431000787EE6600302463E30570302463E76282A
:10432000D2579001F0E014F0E0600302463E7402C0
:10433000F0900096E0900006F0900098E090001059
:10434000F09001E9806C9001E9E0640260030244AE
:1043500010126C37EF6002800C900098E0601090B3
:104360000010E0700A12778B9001E97403F0227854
:104370007EE6600302463E30570302463E9001F05F
:10438000E07033A249924E9001EAE09001B4F090BF
:1043900001EBE09001B5F0900065E09001B6F012FD
:1043A00083749001B7EFF0127E62D23F126E3490A8
:1043B00001F07402F022127B77EF6401704F9001DC
:1043C000B2E0FF249CF582E43401F583E09001B46F
:1043D000F074872FF582E43401F583E09001B5F0A5
:1043E0009001B2E09001B6F012826E9001B7EFF04A
:1043F0009001B4E024DCF582E43400F583E024FF8E
:10440000924E127E62D23F126E340244C00244C009
:104410009001E9E0B4032C206120900223E4F0A392
:1044200074FFF090021F7401F0D26112778BE49058
:1044300001F1F09001E97404F0227BFF7A0F79C951
:104440000246239001E9E064047043787EE660034D
:1044500002463E30570302463EA249924E9001EA80
:10446000E09001B4F09001EBE09001B5F09001B65E
:10447000741FF012001C9001B7EFF0127E629001E1
:10448000F07403F0126E349001E97405F02290018B
:10449000E9E0FF64057030787EE6600302463E3056
:1044A000570302463E9001F0E0700F900097E090B5
:1044B0000001F09001E97406F022787E7628D25748
:1044C0009001F0E014F022EF640660030245C93069
:1044D0005C77304A74C24A900052E0FFC394155092
:1044E0006874DC2FF582E43400F583E0FFA248E431
:1044F000336F7055A2489249900052E09001EAF063
:10450000900053E09001EBF0900051E09001ECF04E
:10451000641F60359001EAE0FFC39415502B74DCF2
:104520002FF582E43400F583E0FFA249E433B507B8
:10453000189001EAE0FF9001EBE0FD7C00127F980B
:104540009001E87402F0024608C24A787EE670558F
:10455000205752127C45EF6401704A9001B2E0FF8F
:10456000249CF582E43401F583E09001B4F0748773
:104570002FF582E43401F583E09001B5F09001B2AB
:10458000E09001B6F012826E9001B7EFF09001B4A6
:10459000E024DCF582E43400F583E024FF924E123F
:1045A0007E62126E34900001E0600302463E12917A
:1045B000A4EF6401600C1277799000BEE0600312F2
:1045C000779D9001E97407F0229001E9E06407709B
:1045D000552061499002237418F0A3E4F090021F63
:1045E00004F0D2619001FDF09000A3E0FF90000E76
:1045F000E4F0A3EFF0900206740FF0E49001E8F00D
:104600001291A4EF64016006E49001E9F022E490C5
:104610000248F0900245F09001E904F0227BFF7A15
:104620000F79DA028F979001E9E0D39407400FE405
:0F4630009001E8F09001E9F090000EF0A3F02265
:1030CE009001E9E070107BFF7A0F79EB128F62901E
:1030DE0001E97401F0229001E9E064017059900059
:1030EE0000E060030235C3A249924E9001EAE090DF
:1030FE0001B4F09001EBE09001B5F0900065E09026
:10310E0001B6F01283749001B7EFF0127E62D23FD7
:10311E00126E34900096E0900006F0900098E090C9
:10312E000010F09000C2E09001FEF09001F07405E6
:10313E00F09001E902329E9001E9E06402702C12D7
:10314E0092C8787EE660030235C33057030235C35A
:10315E007628D2579001F0E014F0E060030235C3F8
:10316E007402F09001E904F0C24A229001E9E06491
:10317E000360030232FC1292C8126C37EF607812B1
:10318E00778B7BFF7A0F79EB128F629000C2E07023
:10319E000302322A128CD3EF64017057304A54C2A4
:1031AE004A900052E0FFC39415504874DC2FF5820C
:1031BE00E43400F583E0FFA248E4336F7035126DFE
:1031CE0092900051E0641F602A9001EAE0FF9000A7
:1031DE0052E0B5071E9001EBE0FF900053E0B507FB
:1031EE00129000C2E09001FEF0C24A900096E0906C
:1031FE000006F0C24A80089000C2E09001FEF02066
:10320E005D0B9000C2E0700512778B800F9000C2AC
:10321E00E060169001FEE0701012778B90020C7435
:10322E0018F09001E97404F022900248E0B4010B0A
:10323E0012778BE4900248F002330D900098E06014
:10324E000C900010E0700612778B02330D787EE63C
:10325E0060030235C33057030235C39001F0E070AE
:10326E0033A249924E9001EAE09001B4F09001EB46
:10327E00E09001B5F0900065E09001B6F012837415
:10328E009001B7EFF0127E62D23F126E349001F0D1
:10329E007402F022127B77EF6401704F9001B2E05E
:1032AE00FF249CF582E43401F583E09001B4F074C0
:1032BE00872FF582E43401F583E09001B5F090019B
:1032CE00B2E09001B6F012826E9001B7EFF090016D
:1032DE00B4E024DCF582E43400F583E024FF924E62
:1032EE00127E62D23F126E340233CA0233CA90018A
:1032FE00E9E0FFB4041090020CE060030235C390C5
:10330E0001E97405F022EFB4052C20612090022310
:10331E00E4F0A374FFF090021F7401F0D2611277F3
:10332E008BE49001F1F09001E97406F0227BFF7AB4
:10333E000F79FC0235A89001E9E064067046787EAC
:10334E00E660030235C33057030235C3A249924EDD
:10335E009001EAE09001B4F09001EBE09001B5F03D
:10336E009001B6741FF012001C9001B7EFF0127EA0
:10337E006212778B9001F07403F0126E349001E9B3
:10338E007407F0229001E9E0FF64077036787EE65C
:10339E0060030235C33057030235C39001F0E0706D
:1033AE0015900097E0900001F09002057432F090B5
:1033BE0001E97408F022787E7628D2579001F0E069
:1033CE0014F022EF6408600302354E900001E070A5
:1033DE0021900205E0701B1291A4EF6401600C12A3
:1033EE0077799000BEE0600312779D9001E9740931
:1033FE00F022787EE67055205752127C45EF64011C
:10340E00704A9001B2E0FF249CF582E43401F5830A
:10341E00E09001B4F074872FF582E43401F583E077
:10342E009001B5F09001B2E09001B6F012826E906C
:10343E0001B7EFF09001B4E024DCF582E43400F53E
:10344E0083E024FF924E127E62126E34128CD3EF02
:10345E0064016003023548204A030235C3C24A1292
:10346E008CD3EF640160030235C39001EAE0FF9054
:10347E000052E0FEB5071A900053E0FF9001EBE01A
:10348E00B5070E900097E0900001F0E49001EEF089
:10349E0022EEC3941540030235C3900052E0FF2480
:1034AE00DCF582E43400F583E0FEA248E4336E607E
:1034BE00030235C39001EEE0FE701AA248924990C5
:1034CE0001EDEFF0900053E09001EEF0900051E02E
:1034DE009001EFF022900052E0FF6E60030235C3C0
:1034EE00A24892499001EAEFF0900053E09001EB70
:1034FE00F0900051E09001ECF0641F70030235C3B0
:10350E009001EAE0FFC3941540030235C374DC2F2B
:10351E00F582E43400F583E0FFA249E4336F6003E3
:10352E000235C39001EAE0FF9001EBE0FD7C001252
:10353E007F989001E87402F08045E4900205F02235
:10354E009001E9E0640970552061499002237418D6
:10355E00F0A3E4F090021F04F0D2619001FDF09010
:10356E0000A3E0FF90000EE4F0A3EFF090020674CB
:10357E000FF0E49001E8F01291A4EF64016006E40C
:10358E009001E9F022E4900248F0900245F090019B
:10359E00E904F0227BFF7A10790D028F979001E9F2
:1035AE00E0D39409400FE49001E8F09001E9F09027
:0635BE00000EF0A3F02254
:104D4E009001E9E07076900065E090005CF09000D4
:104D5E005D74FEF020615C9001F7E0FBB4010FE59D
:104D6E00412400FEE43415900223F0A3CEF0EBB400
:104D7E0002119001F9E02400FEE43416900223F0B3
:104D8E00A3CEF090021F7401F0D261900098E090D3
:104D9E000010F090009BE0900008F090006AE06038
:104DAE000BE49001E9F09001E8024F2D9001E974B7
:104DBE0001F0227BFF7A10791E0250B79001E9E0D4
:104DCE006401707B900000E060030250C9C26090E5
:104DDE0001F7E064017025AF41129248E54175F08C
:104DEE0010A424B8F9741135F0FA7BFF128F62E526
:104DFE004175F010A424B8F9741180359001F7E0D4
:104E0E00640260030250C99001F9E0FF1221529032
:104E1E0001F9E075F010A424F8F9741435F0FA7B5A
:104E2E00FF128F629001F9E075F010A424F8F97466
:104E3E001435F0FA7BFF128F979001E902506E90B5
:104E4E0001E9E064027059126507EF602A206027BD
:104E5E0012778B9000A9E07002803E7BFF7A10796A
:104E6E002F128F979000A9E0900009F0D260900069
:104E7E0067E0700312934C30600A120086500512E0
:104E8E00778B8015900098E070030250C990001047
:104E9E00E060030250C912778B9001E97403F0228F
:104EAE009001E9E0B4032B20611F900223E4F0A3EC
:104EBE0074FFF090021F7401F0D261E49001F8F0DB
:104ECE009001E97404F002934C7BFF7A1079400252
:104EDE0050B79001E9E0B4042D9000AAE060197B70
:104EEE00FF7A107951128F979000AAE0900002F08D
:104EFE009001E97405F0800E900097E0900001F0AB
:104F0E009001E97406F09001E9E0FFB405159000F8
:104F1E0002E0700F900097E0900001F09001E974AC
:104F2E0006F022EF64066003025075900001E070F7
:104F3E00151277799000BEE0600312779DC239900A
:104F4E0001E97407F022205C03024FFD303B44C29E
:104F5E003B9001F7E0B40107E541B5400280479070
:104F6E0001F5E540F0E075F010A424B8F9741135A0
:104F7E00F0FA7BFF128F629001F5E0FF1285F5903B
:104F8E000068E0600E9001F77401F09001F5E0F515
:104F9E00418050304159C2419001F7E0B402109067
:104FAE0001F9E0B53609900097E0900001F02290EB
:104FBE0001F6E536F0E075F010A424F8F974143516
:104FCE00F0FA7BFF128F629001F6E0FF1282F190F1
:104FDE000068E0601A9001F77402F09001F6E0901C
:104FEE0001F9F0E49001E9F09001E87405F022C2B5
:104FFE003BC241128CD3EF64017069304A66129342
:10500E004CC239C24A900052E0FFC39415505574F9
:10501E00DC2FF582E43400F583E0FFA248E4336F21
:10502E007042A2489249900052E09001EAF090003E
:10503E0053E09001EBF0900051E09001ECF0126D16
:10504E00929001ECE0641F601B9001EAE0FF90017A
:10505E00EBE0FD7C00127F98E49001E9F09001E80E
:10506E007402F022C24A229001E9E06407703D20EA
:10507E0061319002237418F0A3E4F090021F04F043
:10508E00D2619001FDF09000A3E0FF90000EE4F0DD
:10509E00A3EFF0900206740FF0E49001E8F0900197
:1050AE00E9F0227BFF7A107962028F979001E9E096
:0C50BE00D394074006E4F09001E8F022D3
:1050CA009001E9E070127BFF7A107973128F629077
:1050DA0001E97401F00277859001E9E064017062E8
:1050EA00900000E06003025443C260900098E09090
:1050FA000010F09000C2E09001FEF09001F7E0B4D9
:10510A000112AF41129248E54175F010A424B8F992
:10511A00741180209001F7E0640260030254439006
:10512A0001F9E0FF1221529001F9E075F010A42470
:10513A00F8F9741435F0FA7BFF128F979001E9029F
:10514A0053E89001E9E0640260030251F81292C840
:10515A00126507EF6033206030D26012778B9000BF
:10516A00A9E0700B12778B9000C2E0701C80507B14
:10517A00FF7A107984128F979000A9E0900009F0C5
:10518A00900067E0700312934C3060401200865022
:10519A00147BFF7A107995128F979000C2E0700DF8
:1051AA0012778B801A9000C2E09001FEF0127D0601
:1051BA009000C2E060169001FEE0701012778B90AA
:1051CA00020C7418F09001E97403F022900248E08E
:1051DA00B40104E4F08012900098E0700302544392
:1051EA00900010E0600302544312778B8011900103
:1051FA00E9E0FFB4031090020CE06003025443900C
:10520A0001E97404F022EFB4042320611790022309
:10521A00E4F0A374FFF090021F7401F0D2619001D0
:10522A00E902536E7BFF7A1079A60254319001E9A4
:10523A00E06405703312934CE49001F8F09000AAF0
:10524A00E060187BFF7A107951128F979000AAE0DC
:10525A00900002F09001E97406F02290020574327F
:10526A00F09001E97407F0229001E9E0FFB4061E0C
:10527A00900002E06003025443900097E09000011E
:10528A00F09001E97407F09002057432F022EF649D
:10529A000760030253EF900001E0701B900205E0E3
:1052AA0070151277799000BEE0600312779DC239BB
:1052BA009001E97408F022205C03025372303B4CDF
:1052CA00C23B9001F7E0B40107E541B54002804FC7
:1052DA009001F5E540F0E075F010A424B8F97411D6
:1052EA0035F0FA7BFF128F629001F5E0FF1285F527
:1052FA00900068E060169001F77401F09001F5E003
:10530A00F541E49001E9F09001E88058304162C229
:10531A00419001F7E0B402109001F9E0B536099026
:10532A000097E0900001F0229001F6E536F0E07572
:10533A00F010A424F8F9741435F0FA7BFF128F6286
:10534A009001F6E0FF1282F1900068E0602390017C
:10535A00F77402F09001F6E09001F9F0E49001E9A7
:10536A00F09001E87405F022C23BC241E4900205C4
:10537A00F0128CD3EF64017069304A6612934CC202
:10538A0039C24A900052E0FFC39415505574DC2F7D
:10539A00F582E43400F583E0FFA248E4336F7042FB
:1053AA00A2489249900052E09001EAF0900053E03E
:1053BA009001EBF0900051E09001ECF0126D9290A8
:1053CA0001ECE0641F601B9001EAE0FF9001EBE052
:1053DA00FD7C00127F98E49001E9F09001E87402E4
:1053EA00F022C24A229001E9E06408703D2061314E
:1053FA009002237418F0A3E4F090021F04F0D26123
:10540A009001FDF09000A3E0FF90000EE4F0A3EFFE
:10541A00F0900206740FF0E49001E8F09001E9F0D0
:10542A00227BFF7A1079B7028F979001E9E0D39433
:0A543A00084006E4F09001E8F022BB
:1035C4009001E9E070212061159002237419F0A3A1
:1035D4007403F090021F7401F0D261023A357BFF4C
:1035E4007A1079C8023A4F9001E9E0B401267BFFD2
:1035F4007A1079D9128F6290005CE024DCF582E4C1
:103604003400F583E024FF9249E4900245F09001F0
:10361400E90239E99001E9E06402704C900000E0AD
:103624006003023A61A249924E9001EAE09001B42B
:10363400F09001EBE09001B5F0900065E09001B6E8
:10364400F01283749001B7EFF0127E62D23F126ED3
:103654003490008CE0900200F0900098E09000100C
:10366400F09001E97403F0229001E9E0640360033F
:103674000237C61292C8126C37EF606F12778B7BD9
:10368400FF7A1079D9128F62128CD3EF64017057CC
:10369400304A54C24A900052E0FFC3941550487413
:1036A400DC2FF582E43400F583E0FFA248E4336FB5
:1036B4007035126D92900051E0641F602A9001EA07
:1036C400E0FF900052E0B5071E9001EBE0FF900090
:1036D40053E0B5071290008CE0900200F0C24A90CB
:1036E4000096E0900006F0C24A800890008CE090BA
:1036F4000200F0900248E0B40104E4F0801A900261
:1037040000E0700890008CE06002800C900098E06B
:103714006010900010E0700A12797B9001E9740443
:10372400F022787EE66003023A61305703023A6180
:103734009001F0E07032A249924E9001EAE09001CB
:10374400B4F09001EBE09001B5F0900065E09001D9
:10375400B6F01283749001B7EFF0127E62D23F127A
:103764006E349001F00239E9127B77EF6401704FF7
:103774009001B2E0FF249CF582E43401F583E090EB
:1037840001B4F074872FF582E43401F583E09001ED
:10379400B5F09001B2E09001B6F012826E9001B7DC
:1037A400EFF09001B4E024DCF582E43400F583E02A
:1037B40024FF924E127E62D23F126E3402387B0294
:1037C400387B9001E9E0B4042620611A900223E4D6
:1037D400F0A374FFF090021F7401F0D2619001E92C
:1037E4007405F002778B7BFF7A1079EA023A4F90E6
:1037F40001E9E06405704812778B787EE660030285
:103804003A61305703023A61A249924E9001EAE0CC
:103814009001B4F09001EBE09001B5F09001B67422
:103824001FF012001C9001B7EFF0127E62D23F909D
:1038340001F07403F0126E349001E97406F02290E2
:1038440001E9E0FF64067036787EE66003023A61BF
:10385400305703023A619001F0E07015900097E050
:10386400900001F09002057432F09001E97407F0C1
:1038740022787E7628D2579001F0E014F022EF648B
:103884000760030239F5900001E0701B1291A4EF68
:103894006401600C1277799000BEE0600312779D9A
:1038A4009001E97408F022787EE670552057521290
:1038B4007C45EF6401704A9001B2E0FF249CF582DC
:1038C400E43401F583E09001B4F074872FF582E4C9
:1038D4003401F583E09001B5F09001B2E09001B6B7
:1038E400F012826E9001B7EFF09001B4E024DCF5A1
:1038F40082E43400F583E024FF924E127E62126E5D
:1039040034128CD3EF640160030239ED204A0302C0
:1039140039F212934CC239C24A9001EAE0FF900096
:1039240052E0FEB5071A900053E0FF9001EBE0B5BA
:10393400070E900097E0900001F0E49001EEF02271
:10394400EEC3941540030239F2900052E0FF24DCE8
:10395400F582E43400F583E0FEA248E4336E6003AC
:103964000239F29001EEE0FE701BA24892499001E8
:10397400EDEFF0900053E09001EEF0900051E090F4
:1039840001EFF08069900052E0FF6E7061A24892EE
:10399400499001EAEFF0900053E09001EBF09000C1
:1039A40051E09001ECF0126D929001ECE0641F6024
:1039B4003D9001EAE0FFC39415503374DC2FF58287
:1039C400E43400F583E0FFA249E433B50720900115
:1039D400EAE0FF9001EBE0FD7C00127F98E49001A7
:1039E400E9F09001E87402F022E4900205F0C24A82
:1039F400229001E9E0640870552061499002237423
:103A040018F0A3E4F090021F04F0D2619001FDF0DD
:103A14009000A3E0FF90000EE4F0A3EFF090020604
:103A2400740FF0E49001E8F01291A4EF64016006D1
:103A3400E49001E9F022E4900248F0900245F0900D
:103A440001E904F0227BFF7A1079FB028F97900141
:0E3A5400E9E0D394084006E4F09001E8F02287
:10463F009001E9E0703F900065E090005CF0900021
:10464F005D74FEF02061259001F7E0900223B40124
:10465F00097419F0A37401F080077419F0A37402A0
:10466F00F090021F7401F0D2610249AC7BFF7A1106
:10467F00790C128F979001E9E06401702C9001F78B
:10468F00E07BFFB4010E7A11791D128F62AF4112D8
:10469F0085F5800F7A117930128F629001F9E0FF62
:1046AF001282F19001E902496E9001E9E064027013
:1046BF006C305C05127785800312778B900000E0D9
:1046CF0060030249C990008CE0900200F0900098BE
:1046DF00E0900010F09001F7E0B40112AF41129298
:1046EF0048E54175F010A424B8F9741180209001A9
:1046FF00F7E0640260030249C99001F9E0FF12215B
:10470F00529001F9E075F010A424F8F9741435F003
:10471F00FA7BFF128F979001E97403F0229001E961
:10472F00E06403707C1292C8305C3C9001F7E0B4F7
:10473F000115303B12E541B5400D90008CE0900221
:10474F0000F0C23B1277859001F7E0B402203041B0
:10475F001D9001F9E0B5361690008CE0900200F044
:10476F00C241127785800712778BC23BC2419002FC
:10477F0048E0B401028020900200E0700890008CA5
:10478F00E060028012900098E070030249C9900027
:10479F0010E060030249C912797B9001E97404F0BB
:1047AF00229001E9E0B40423206117900223E4F082
:1047BF00A374FFF090021F7401F0D2619001E9021F
:1047CF0048FE7BFF7A1179410249B79001E9E06415
:1047DF0005702712778B12934C9000AAE060307B04
:1047EF00FF7A107951128F979000AAE0900002F093
:1047FF0012934C9001E97406F0229001E9E0B4069F
:10480F0015900002E0700F900097E0900001F0907B
:10481F0001E97407F0229001E9E06407600302499F
:10482F0075900001E070131277799000BEE060037D
:10483F0012779D9001E97408F022205C030249026F
:10484F00303B4EC23B9001F7E0B40109E5416540B2
:10485F0070030249C99001F5E540F0E075F010A42E
:10486F0024B8F9741135F0FA7BFF128F629001F5BD
:10487F00E0FF1285F5900068E060169001F7740173
:10488F00F09001F5E0F541E49001E9F09001E88046
:10489F005E30415FC2419001F9E536F09001F7E0DB
:1048AF00B4020B9001F9E0653670030249C990011B
:1048BF00F6E536F075F010A424F8F9741435F0FA13
:1048CF007BFF128F629001F6E0FF1282F19001F7E9
:1048DF007402F0900068E0601A9001F77402F09093
:1048EF0001F6E09001F9F0E49001E9F09001E8742D
:1048FF0005F022C23BC241305C69304A6612934CCC
:10490F00C239C24A900052E0FFC39415505574DC6F
:10491F002FF582E43400F583E0FFA248E4336F7093
:10492F0042A2489249900052E09001EAF090005361
:10493F00E09001EBF0900051E09001ECF0126D92DD
:10494F009001ECE0641F601B9001EAE0FF9001EB27
:10495F00E0FD7C00127F98E49001E9F09001E8748B
:10496F0002F022C24A229001E9E06408703D206102
:10497F00319002237418F0A3E4F090021F04F0D2D8
:10498F00619001FDF09000A3E0FF90000EE4F0A312
:10499F00EFF0900206740FF0E49001E8F09001E957
:1049AF00F0227BFF7A117952028F979001E9E0D3C1
:0B49BF0094084006E4F09001E8F022AC
:105AD7009001E9E0FF70362061339002237418F0DB
:105AE700A37401F090021FF0D2619000BFE0FE6442
:105AF700016004EEB402079001E97401F022EE643C
:105B0700036004EEB404069001E9025CAFEF6401A0
:105B17006003025C06128CD3BF010890009DE090E1
:105B27000005F0900005E0700F1277799000BEE055
:105B3700600312779D025C319000BFE0B401097BDE
:105B4700FF7A117963025C521277739000BEE060AE
:105B5700031277977BFF7A117974128F62787EE64A
:105B67006003025D47305703025D479001F0E07024
:105B770034D23F9000A4E024FF924E900065E0FFEE
:105B87009001B4F09000A2E09001B5F09001B6EF5B
:105B9700F01283749001B7EFF0127E62126E3490A8
:105BA70001F0025CAF127B77EF6401704FD23F9038
:105BB70001B2E0FF249CF582E43401F583E0900113
:105BC700B4F074872FF582E43401F583E09001B5D2
:105BD700F09001B2E09001B6F012826E9001B7EF3B
:105BE700F09001B4E024DCF582E43400F583E0248E
:105BF700FF924E127E62126E34025D09025D0990B9
:105C070001E9E064026003025D10129057BF0108CA
:105C170090009DE0900005F0900005E0702012775D
:105C2700799000BEE0600312779D9000A3E0FF909B
:105C3700000EE4F0A3EFF09001E97403F022900066
:105C4700BFE0B403097BFF7A117985028F6212776F
:105C5700739000BEE060031277977BFF7A11799605
:105C6700128F62787EE66003025D47305703025D5C
:105C7700479001F0E07035D23F9000A4E024FF92F6
:105C87004E900065E0FF9001B4F09000A2E0900113
:105C9700B5F09001B6EFF01283749001B7EFF012F0
:105CA7007E62126E349001F07402F022127B77EF5D
:105CB7006401704ED23F9001B2E0FF249CF582E46C
:105CC7003401F583E09001B4F074872FF582E43452
:105CD70001F583E09001B5F09001B2E09001B6F0D4
:105CE70012826E9001B7EFF09001B4E024DCF582E8
:105CF700E43400F583E024FF924E127E62126E3484
:105D070080009001F0E014F0229001E9E0B4031E56
:105D17002061129002237418F0A3E4F090021F048C
:105D2700F0D26180127BFF7A1179A7128F979001C9
:105D3700E9E0D394034009E49001E8F09001E9F029
:015D47002239
:0D008600900009E07002D322127D06C32213
:107D0600205C03027DA89001F7E064017040303BDF
:107D16003DC23BE54165407035C260AF41129248B5
:107D2600E54175F010A424B8F9741135F0FA7BFF1B
:107D3600128F62E54175F010A424B8F9741135F07C
:107D4600FA7BFF128F9790009BE0900008F090015D
:107D5600F7E06402705A304157C2419001FAE536A5
:107D6600F09001F9E0FF65367046C260122152902C
:107D760001F9E075F010A424F8F9741435F0FA7BD3
:107D8600FF128F629001F9E075F010A424F8F974DF
:107D96001435F0FA7BFF128F9790009BE090000855
:107DA600F022E47888F608F608F608F6C23BC241E7
:017DB60022AA
:1000A600202020202020202020202020202020204A
:1000B6005245504541544552204E554D42455220D9
:1000C6002020202020202020203120746F20323054
:1000D600202053495445204E554D4245522020205C
:1000E6002020202020202020203120746F20393924
:1000F6008202001101021501148202011103041586
:1001060001632020202020202020202020202020C5
:1001160020202020202020202020202020202020D9
:10012600202020434F5552544553592042454550AF
:100136002020204354435353204F4E2048414E47DE
:10014600202020205553455220454E41424C452003
:10015600202020205245534552564520544F4E45A7
:10016600202020204E4554574F524B204D4F44459A
:100176002020204E4554574F524B204E554D424558
:100186005220202020202020202020202020202037
:100196002020202020202020202020202020202059
:1001A6002020202020202020202020202020202049
:1001B6002020202020202020202020202020202039
:1001C6002020202020202020202020202020313DFB
:1001D600454E2020202020202020202020204D4F6A
:1001E6004445202020202020202020202020544F5D
:1001F6004E4564010011020C150001640200110352
:100206000C15000164040011040C150001640800BB
:1002160011050C15000164100011060D150002C829
:10022600030111070A190101202020202020202087
:1002360020202020202020202020202020202020B8
:10024600202020202020202020434F555254455363
:100256005920424545502020204354435353204FB4
:100266004E2048414E4720202020555345522045D8
:100276004E41424C4520202020205245534552569F
:100286004520544F4E45202020204E4554574F526E
:100296004B204D4F44452020204E4554574F524B3E
:1002A600204E554D4245522020202020202020203F
:1002B6002020202020202020202020202020202038
:1002C6002020202020202020202020202020202028
:1002D6002020202020202020202020202020202018
:1002E6002020202020202020202020202020202008
:1002F60020202020313D454E202020202020202077
:10030600202020204D4F4445202020202020202042
:1003160020202020544F4E4564010011020C150088
:100326000164020011030C15000164040011040CA1
:1003360015000164080011050C1500016410001178
:10034600060D150001C8030111070A190101202035
:100356002020202020202020202020202020202097
:100366002020202020202020202020202020204364
:100376004F55525445535920424545502020202080
:100386005553455220454E41424C4520202020439E
:10039600524F535320544F4E45204D4F4445204312
:1003A600544353532F4443532043524F5353202017
:1003B6004E4554574F524B204D4F44452020204E1A
:1003C6004554574F524B204E554D42455220202002
:1003D6002020202020202020202020202020202017
:1003E60020202020202020202020313D454E202086
:1003F600202020202020202020204D4F4445202052
:1004060020202020202020202020544F4E45202030
:1004160020202020202020202020202020206401B1
:1004260000110209150001640200110309150001FB
:1004360064040011060A150001C8030111070C190E
:1004460001012020202020202020202020202020E4
:100456002020202020202020202020202020202096
:10046600202001010101010101010100000000003D
:100476000000000000000000000000000000000076
:100486000000000000000000000000000000000066
:100496000000000000000000000000000000000056
:1004A6000000000000000000000000000000000046
:1004B60000000000000000000000000020202020B6
:1004C6002020202020202020202020202020202026
:1004D6002020202020202020202020200101010192
:1004E6000101010101000000000000000000000001
:1004F60000000000000000000000000000000000F6
:1005060000000000000000000000000000000000E5
:1005160000000000000000000000000000000000D5
:1005260000000000000000000000000000000000C5
:100536000000000000002020202020202020202075
:1005460020202020202020202020202020202020A5
:1005560020202020202001010101010101010120AC
:100566002020202020202020202020202020202085
:100576002020202020202020202020202020202075
:1005860054454C434F2050524F4752414D20202056
:10059600524144494F2050524F4752414D2020204E
:1005A60050484F4E452050524F4752414D20202033
:1005B600434F4D50552050524F4752414D20202019
:1005C6002041434345535320434F44452020204474
:1005D600544D462054454C434F204C4556454C44BB
:1005E600544D4620524144494F204C4556454C42B5
:1005F60045455020524144494F204C4556454C42B2
:100606004545502054454C434F204C4556454C4398
:1006160057494420524144494F204C4556454C5673
:100626004F49434520524144494F204C45564C566C
:100636004F4943452054454C434F204C45564C505A
:1006460041474520524144494F204C4556454C436D
:100656005443535320524144494F204C45564C4431
:10066600435320524144494F204C4556454C204C5B
:10067600545220524144494F204C4556454C205235
:10068600505420524144494F204C4556454C205425
:10069600454C434F20524144494F204C45564C52FD
:1006A6004144494F2054454C434F204C45564C52EB
:1006B6004144494F204C494D4954204C45564C2005
:1006C600434F53204F5220535155454C4348202009
:1006D60020434F5320504F4C4152495459202043F8
:1006E6004F53205452494747455220564F4C544386
:1006F6004F5320414351554953542054494D454386
:100706004F532052454C454153452054494D4520B1
:1007160053454E534520504F4C415249545920534E
:10072600454E205452494747455220564F4C545344
:10073600454E20414351554953542054494D455344
:10074600454E2052454C454153452054494D452080
:100756004C545220484F4C442044454C415920505B
:100766005454205455524E4F46462054494D4552F6
:10077600455045415445522054494D454F55542006
:1007860020414E54492D4B45524348554E4B20204F
:1007960020535155454C4348205441494C20202074
:1007A60043544353532F44435320484F4C44204310
:1007B600524F535320425553592044454C415943B7
:1007C600524F5353204255535920484F4C442020F2
:1007D600204C54522053594E432042495420202045
:1007E600414456414E43454420204C4F434B202024
:1007F60020202020202020202020202020202020F3
:1008060020202020202020202020202020202020E2
:1008160020202020202020202020202020202020D2
:1008260020202020202020202020202020202020C2
:100836002020202020202020202020313D454E2031
:1008460020202020202020202020524154494F20C3
:1008560020202020202020202020303D434F5320E0
:1008660020202020202020202020313D504F5320C2
:10087600202020202020202020202031204D532001
:10088600202020202020202020203130204D5320E1
:10089600202020202020202020313030204D5320C1
:1008A60020202020202020202020202053454320C7
:1008B600202020202020202020313D534B4950204D
:1008C6002020202020202020202020202020202022
:1008D6002020202020202020202020202020202012
:1008E6005052494F52495459204C4556454C2020A8
:1008F6004C545220454E434F444520504F4C2020E7
:100906004C5452204445434F444520504F4C2020E0
:10091600205445535420494420434F444520204900
:10092600444C45204D45535341474520544D522094
:100936002020204152454120424954202020202099
:100946004D4153544552204F5220534C4156452059
:1009560044435320454E434F444520504F4C20209E
:10096600444353204445434F444520504F4C202098
:10097600434F5552544553592044454C4159202024
:10098600202048414E472054494D452020202043F1
:100996004152524945522044524F5020444C59200E
:1009A600204143434553532044454C41592020534D
:1009B600544154494F4E204944204D4F4445202030
:1009C600564F494345204F52204357494420202043
:1009D60020494420494E54455256414C202020205F
:1009E6002020435749442053504545442020202089
:1009F60043574944204652455155454E43592020B8
:100A06002043574944204D45535341474520202014
:100A16005455524E5F4F4E2044454C41592020209C
:100A26005455524E5F4F46462044454C415920206E
:100A360042454550204652455155454E4359205250
:100A4600455045415445522044495341424C452066
:100A56004155582052454C4159204D4F4445202080
:100A660043524F53532042555359204D4F4445202E
:100A76005245504541544552204741494E20202079
:100A86002054454C434F204741494E202020204EBC
:100A96004554574F524B2048414E4754494D4520E7
:100AA6002020202020202020204C4556454C202068
:100AB600202020202020202020303D4E4F524D2047
:100AC6002020202020202020202020434F44452085
:100AD6002020202020202020202020415245412077
:100AE60020202020202020303D4D415354455220C7
:100AF600202020202020202020202031204D53207F
:100B0600202020202020202020203130204D53205E
:100B1600202020202020202020313030204D53203E
:100B26002020202020202020203130205345432023
:100B36002020202020202020202031204D494E201A
:100B460020202020202020202020204D4F444520FA
:100B56002020202020202020303D564F494345208C
:100B660020202020202020202020204652455120D1
:100B76002020202020202020202020313D454E20EE
:100B860020414C41524D20434F554E5420202020A9
:100B9600524553544F524520434F554E5420202022
:100BA6002020494E54455256414C202020202020DA
:100BB6004E4554574F524B20434F44452020204921
:100BC6004E544552434F4E4E454354204D4F444E8E
:100BD6004554574F524B20494E414354495645823E
:100BE600010011022D15000182010111032D1500CE
:100BF6000182010211042D15000182010311052D48
:100C060015000178060411060119010182030A1173
:100C1600072E1500FF82030B11082E1500FF820315
:100C26000C11092E1500FF82030D110A2E1500FF67
:100C360082030E110B2E1500FF82030F110C2E15C9
:100C460000FF820310110D2E1500FF820311110EF5
:100C56002E1500FF820312110F2E1500FF820313BB
:100C660011102E1500FF82031411112E1500FF829C
:100C7600031511122E1500FF82031611132E1500EF
:100C8600FF82031711142E1500FF82031811152E6B
:100C96001500FF82011911162F15000182011A1184
:100CA600173015000182031B11182E1500FF820252
:100CB6001C11193115006382021D111A32150063C9
:100CC60082011E111B3015000182031F111C2E15F7
:100CD60000FF820220111D31150063820221111EC0
:100CE60032150063820222111F3315026382032329
:100CF6001120321501FF8203241121341502FF82CF
:100D060002251122331500638202261123321500B3
:100D160063820227112433150363820228112532C8
:100D26001500638203291126331500FA82012A1160
:100D3600273515000182012B11385415010982014E
:100D46002C11395515000182012D113A5515000156
:100D560082032E113B561501FA82032F113C5C15B6
:100D660000FF820130113D57150001820131113E0D
:100D760058150001820132113F55160001820133D8
:100D860011405515000182023411415A1500638243
:100D9600023511425B15006382023611435A150073
:100DA6006382023711445A15006382013811455E89
:100DB60015000182013911465F15000182023A11C0
:100DC600475D15006382023B114859150463820290
:100DD6003C114960150114BE0A3D114A5611000026
:100DE600820247114B5A150063820248114D601565
:100DF6000114820149114E5E15000282014A114F0B
:100E06006115000182014B11505E15000482014CF0
:100E160011515415010982014D11525415010982CF
:100E2600024E11533415006382014F116201150001
:100E36000982015011630115000982025111645D96
:100E4600150163C803521165011501018201541190
:100E5600665E1500028203551167341500FF010115
:100E66000200000200000200000000000001010173
:100E76003132333435361432320532FFFFFF191959
:100E8600196464C8FF000180000A0180000A1E1A66
:100E9600B400001E1E1E0001000002010001000039
:100EA6000A1E630A000100050520202020202020BC
:100EB6002020200A050000000101140000010000A6
:020EC60000002A
:108F62008B6E8A6F89707F01127961E4900141F002
:108F7200900141E0FFC39410501AAB6EAA6FA97022
:108F82008F8275830012850FFF127932900141E0C2
:058F920004F080DC2268
:10668C008B6E8A6F8970900252E0B4110040030245
:10669C0068099066A5F82828730266D80266E0029D
:1066AC0066F002670302671602672902673C0267FD
:1066BC004F0267620267750267870267990267ABD0
:1066CC000267BD0267CF0267E10267F37F011279AF
:1066DC0061026803AB6EAA6FA9701284F6FF12797F
:1066EC0032026803AB6EAA6FA97090000112850F7D
:1066FC00FF127932026803AB6EAA6FA97090000288
:10670C0012850FFF127932026803AB6EAA6FA97063
:10671C0090000312850FFF127932026803AB6EAA48
:10672C006FA97090000412850FFF12793202680372
:10673C00AB6EAA6FA97090000512850FFF1279320B
:10674C00026803AB6EAA6FA97090000612850FFF4A
:10675C00127932026803AB6EAA6FA970900007120F
:10676C00850FFF127932026803AB6EAA6FA9709085
:10677C00000812850FFF127932807CAB6EAA6FA9CC
:10678C007090000912850FFF127932806AAB6EAAE5
:10679C006FA97090000A12850FFF1279328058ABE6
:1067AC006EAA6FA97090000B12850FFF12793280C0
:1067BC0046AB6EAA6FA97090000C12850FFF127970
:1067CC00328034AB6EAA6FA97090000D12850FFF4A
:1067DC001279328022AB6EAA6FA97090000E1285CE
:1067EC000FFF1279328010AB6EAA6FA97090000F58
:0E67FC0012850FFF127932900252E004F02253
:108F97008B6E8A6F89707F11127961E4900141F0BD
:108FA700900141E0FFC39410501AAB6EAA6FA970ED
:108FB7008F8275830012850FFF127932900141E08D
:058FC70004F080DC2233
:103E9F00E4900208F0A3F090020AF0900145F0A31D
:103EAF00F0900146E02400F582E43404F583E4F059
:103EBF00900146E004F07006900145E004F0900197
:103ECF0045E07004A3E0648070D7E4900141F09066
:103EDF000141E0FFC394024003023F70EF900E6474
:103EEF0093FF90020AE0FE04F074002EF582E43492
:103EFF0004F583EFF090020AE06480705B90020893
:103F0F00E0FEA3E07807C333CE33CED8F9FF7C04AD
:103F1F007D00127215E4900145F0A3F0900146E088
:103F2F002400F582E43404F583E4F0900146E004C4
:103F3F00F07006900145E004F0900145E07004A395
:103F4F00E0648070D7E490020AF0900209E004F078
:103F5F007006900208E004F0900141E004F0023E88
:103F6F00DEE4900144F0E4900142F0A3F0E490010C
:103F7F0041F0900141E0FFC394034003024013EF6F
:103F8F00900E6693FF90020AE0FE04F074002EF587
:103F9F0082E43404F583EFF090020AE06480705BF2
:103FAF00900208E0FEA3E07807C333CE33CED8F9F2
:103FBF00FF7C047D00127215E4900145F0A3F09090
:103FCF000146E02400F582E43404F583E4F0900127
:103FDF0046E004F07006900145E004F0900145E0E2
:103FEF007004A3E0648070D7E490020AF090020995
:103FFF00E004F07006900208E004F0900141E00444
:10400F00F0023F81900143E004F07006900142E01E
:10401F0004F0C3900143E09433900142E0940050C8
:10402F0003023F7C900144E004F0E0C3941450037A
:10403F00023F75E4900144F0E4900142F0A3F0E4F4
:10404F00900141F0900141E0FFC39403400302400F
:10405F00E5EF900E6993FF90020AE0FE04F0740002
:10406F002EF582E43404F583EFF090020AE06480C9
:10407F00705B900208E0FEA3E07807C333CE33CE27
:10408F00D8F9FF7C047D00127215E4900145F0A36E
:10409F00F0900146E02400F582E43404F583E4F067
:1040AF00900146E004F07006900145E004F09001A5
:1040BF0045E07004A3E0648070D7E490020AF090AA
:1040CF000209E004F07006900208E004F09001414C
:1040DF00E004F0024053900143E004F070069001B9
:1040EF0042E004F0C3900143E09470900142E094E9
:1040FF0000500302404E900144E004F0E0C39414DA
:10410F005003024047E4900142F0A3F0E4900141D4
:10411F00F0900141E0FFC3940340030241B2EF90DE
:10412F000E6C93FF90020AE0FE04F074002EF582ED
:10413F00E43404F583EFF090020AE06480705B9042
:10414F000208E0FEA3E07807C333CE33CED8F9FFE1
:10415F007C047D00127215E4900145F0A3F09001EC
:10416F0046E02400F582E43404F583E4F090014640
:10417F00E004F07006900145E004F0900145E07016
:10418F0004A3E0648070D7E490020AF0900209E083
:10419F0004F07006900208E004F0900141E004F092
:1041AF00024120900143E004F07006900142E004C8
:1041BF00F0C3900143E09488900142E094135003C0
:1041CF0002411B8000E4900142F0A3F0E490014112
:1041DF00F0900141E0FFC394564003024272EF900A
:1041EF000E7293FF90020AE0FE04F074002EF58227
:1041FF00E43404F583EFF090020AE06480705B9082
:10420F000208E0FEA3E07807C333CE33CED8F9FF20
:10421F007C047D00127215E4900145F0A3F090012B
:10422F0046E02400F582E43404F583E4F09001467F
:10423F00E004F07006900145E004F0900145E07055
:10424F0004A3E0648070D7E490020AF0900209E0C2
:10425F0004F07006900208E004F0900141E004F0D1
:10426F000241E0900143E004F07006900142E00447
:10427F00F0C3900143E09414900142E09400500386
:10428F000241DB900208E0FEA3E07807C333CE3390
:10429F00CED8F9FF7C047D0012721512797B02795A
:0142AF008A84
:1090DD00E4900063F0A3F090006375F001128560D9
:1090ED00AFF0FE1271BE900065EFF0900063E0FEF0
:0C90FD00A3E0FF1271BE900207EFF0220A
:107EFD00755501755600755774E490024FF0A3F057
:107F0D0090024FE0FAA3E0FBC39456EA9400504070
:107F1D00900065E075F056A42478FFE5F03460CF4D
:107F2D002BCF3AFE900063F0A3EFF01271BEAB556C
:107F3D000557E557AA567002055614F9EF12853C00
:107F4D00900250E004F070B890024FE004F080B061
:107F5D009000A5E07004D2588002C2589000A1E0B4
:107F6D0024FF92509000A0E024FF92449000A7E0DF
:107F7D0024FF924F9000A6E024FF924590009EE0D2
:0A7F8D0024FF923C900086E0F52DE1
:017F970022C7
:1089B8007555017556007557C9E490024FF0A3F03C
:1089C80090024FE0FEA3E0FFC39414EE9400503BE6
:1089D8007C007D5612854EEF24F9FFEE3460FE9040
:1089E8000063F0A3EFF01271BEAB550557E557AA27
:1089F800567002055614F9EF12853C900250E004B7
:0B8A0800F070BD90024FE004F080B55C
:018A13002240
:108A14007555017556007557DDE490024FF0A3F0CB
:108A240090024FE0FEA3E0FFC39414EE9400503B89
:108A34007C007D5612854EEF24FEFFEE3460FE90DE
:108A44000063F0A3EFF01271BEAB550557E557AACA
:108A5400567002055614F9EF12853C900250E0045A
:0B8A6400F070BD90024FE004F080B500
:018A6F0022E4
:1085F5008F6EE4900141F0900141E0FBC39403507C
:108605003E900065E075F099A42469FDE5F034FF1E
:10861500FCE56E75F003A42DFFE5F03CFEEB7C0058
:108625002FFFEC3EFE1271BE900141E0246BF582F6
:10863500E43400F583EFF0900141E004F080B89058
:10864500006BE0FE5401900066F0EE540290006766
:10865500F090006BE05404900068F0EE5408900030
:0D86650069F090006BE0541090006AF02264
:1082F1008F6EE4900141F0900141E0FBC394035083
:1083010044900065E0FF7E007C017D5012854EEFB8
:1083110024A6FDEE340AFCE56E75F003A42DFFE5FD
:10832100F03CFEEB7C002FFFEC3EFE1271BE900193
:1083310041E0246BF582E43400F583EFF0900141D4
:10834100E004F080B290006BE0FE5401900066F012
:10835100EE5402900067F090006BE05404900068C6
:10836100F0EE5408900069F090006BE0541090001A
:038371006AF0228D
:067F98008F6E8C6F8D70EE
:107F9E00E490024FF0A3F0E57024FFFFE56F34FF8D
:107FAE00FE7C007D0312854EAA06AB07AE6EE56E13
:107FBE0025E0CE75F0EEA4FFE5F02EFEEF2448FF8F
:107FCE00EE3423CF2BCF3AFE900250E02FFF9002DB
:107FDE004FE03EFE1271BE900250E0246BF582E43B
:107FEE003400F583EFF0900250E004F0700690023A
:107FFE004FE004F0C3900250E0940390024FE094DF
:10800E0000409490006BE0FE5401900071F0EE542D
:0F801E0002900072F090006BE05404900073F039
:01802D002230
:109209002020202020534C4156452020202020207A
:1092190020202020204D4153544552202020202039
:0E935B0012788F12797B12798A7F0102796174
:10902900900003740AF0900003E070FA9000A5E044
:109039007BFF60067A92790980047A927919128FF6
:0E90490097900003740AF0900003E070FA2282
:1073F600C0D0C0E0C0F0C000A88475840FE50A5470
:1074060007B4000D85E8F0A2F09220A2F192218047
:1074160076B4010D85E8F0A2F09222A2F1922380C3
:1074260066B4020D85E8F0A2F09224A2F1922580BE
:1074360056B4030D85E8F0A2F09226A2F1922780B9
:1074460046B4040D85E8F0A2F09218A2F1921980D4
:1074560036B4050D85E8F0A2F0921AA2F1921B80CF
:1074660026B4060D85E8F0A2F0921CA2F1921D80CA
:107476001685E8F0A2F0921EA2F1921F750AFF850A
:107486002331852432D264050A750B0A8884D0001C
:10749600D0F0D0E0D0D03220630122D2B7E50C5430
:1074A60007B4000AA22F92F7A22E92F6805EB401CC
:1074B6000AA22D92F7A22C92F68051B4020AA22BB0
:1074C60092F7A22A92F68044B4030AA22992F7A25E
:1074D6002892F68037B4040AA23792F7A23692F6BB
:1074E600802AB4050AA23592F7A23492F6801DB41A
:1074F600060AA23392F7A23292F68010B40721A2AE
:107506003192F7A23092F6C263750CFF050C7584B2
:107516000F85E8E0A2F692E6A2F792E7F5E8C2B791
:017526002242
:105D48002020204453502052657365742020202061
:105D58000000000000000004000000080000000C23
:105D68000000001000000014000000180000001CD3
:105D78000000002000000024000000280000002C83
:105D88000000003000000034000000380000003C33
:105D98000000004000000044000000480000004CE3
:105DA8000000005000000054000000580000005C93
:105DB8000000006000000064000000680000006C43
:105DC8000000007000000074000000780000007CF3
:105DD8000000108000001084000010880000108C63
:105DE8000000109000001094000010980000109C13
:105DF800000010A0000010A4000010A8000010ACC3
:105E0800000010B0000010B4000010B8000010BC72
:105E1800000010C0000010C4000010C8000010CC22
:105E2800000010D0000010D4000010D8000010DCD2
:105E3800000010E0000010E4000010E8000010EC82
:105E4800000010F0000010F4000010F8000010FC32
:105E58000000218000002184000021880000218C9E
:105E68000000219000002194000021980000219C4E
:105E7800000021A0000021A4000021A8000021ACFE
:105E8800000021B0000021B4000021B8000021BCAE
:105E9800000021C0000021C4000021C8000021CC5E
:105EA800000021D0000021D4000021D8000021DC0E
:105EB800000021E0000021E4000021E8000021ECBE
:105EC800000021F0000021F4000021F8000021FC6E
:105ED8000000318000003184000031880000318CDE
:105EE8000000319000003194000031980000319C8E
:105EF800000031A0000031A4000031A8000031AC3E
:105F0800000031B0000031B4000031B8000031BCED
:105F1800000031C0000031C4000031C8000031CC9D
:105F2800000031D0000031D4000031D8000031DC4D
:105F3800000031E0000031E4000031E8000031ECFD
:105F4800000031F0000031F4000031F8000031FCAD
:015F58000048
:1054440090020EE0FFEF707C900220E0FFEFD39417
:105454000340030257A22064030257A2C2649002CD
:1054640004741EF090021DE531F0A3E532F09002C1
:105474001DE0FEA3E0FFEE541FFE900217EEF0A322
:10548400EFF090021DE0FEA3E0FFEEC4135407FF0B
:105494007E0090021DEEF0A3EFF090021EE0FF905C
:1054A4000210EFF090020FE4F090021DE0FEA3E082
:1054B400FFEF4E7004D262222290021EE0FF90029F
:1054C4000EEFF02290020EE0FFEFB4011A20640305
:1054D4000257A2900219E531F0A3E532F0C264D27A
:1054E4006290020EE4F02290020EE0FFEF6402707C
:1054F400432064030257A2C26490020FE0FFEF70DE
:1055040011900219E531F0A3E532F090020FE004A6
:10551400F02290020FE0FFEFB4011290021BE5317C
:10552400F0A3E532F0D26290020EE4F02290020E73
:10553400E4F0222290020EE0FFEF640360030256BF
:10554400542064030257A2C26490020FE0FFEF707C
:1055540029900219E531F0A3E532F0900215E4F048
:10556400A3E4F0900211E4F0A3E4F0900213E4F059
:10557400A3E4F090020FE004F02290020FE0FFEFAA
:105584006401707990021DE531F0A3E532F09002D8
:105594001DE0FEA3E0FF900212E02FF0900211E064
:1055A4003EF090021DE0FCA3E0FD900213E475F0D0
:1055B40001128560AFF0FEEF25E0FFEE33FE7400CC
:1055C4002FF58274043EF583ECF0A3EDF0900216FF
:1055D400E004F07006900215E004F0900217E0FE7B
:1055E400A3E0FF900215E0FCA3E0FDED6F7002EC78
:1055F4006E60030257A290020F7402F02290020F11
:10560400E0FFEF6402704290021BE531F0A3E53243
:10561400F090020EE4F0900211E0FEA3E0FF90028D
:105624001BE0FCA3E0FDEDB50717ECB506139002F3
:1056340019E0FEA3E0FF1290847F007E901293078E
:10564400227F017E901293072290020EE4F0222220
:1056540090020EE0FFEF6404600302578D206403A0
:105664000257A2C26490020FE0FFEF702990021962
:10567400E531F0A3E532F0900215E4F0A3E4F090F4
:105684000211E4F0A3E4F0900213E4F0A3E4F09038
:10569400020FE004F02290020FE0FFEF6401707348
:1056A40090021DE531F0A3E532F090021DE0FEA367
:1056B400E0FF900212E02FF0900211E03EF0900221
:1056C4001DE0FCA3E0FD900213E475F00112856077
:1056D400AFF0FEEF25E0FFEE33FE74002FF5827489
:1056E400043EF583ECF0A3EDF0900216E004F070B4
:1056F40006900215E004F0900215E0FEA3E0FFEF2F
:1057040064007003EE640260030257A290020FE08B
:1057140004F02290020FE0FFEF6402706590024AE9
:105724007455F090021BE531F0A3E532F0900211BC
:10573400E0FEA3E0FF90021BE0FCA3E0FDEDB50753
:105744002AECB50626900217E0FEA3E0FF12799931
:105754007F007E90129307900219E0FEA3E0FFEF12
:105764004E601990024B74AAF0801190024AE4F042
:1057740090024BE4F07F017E9012930790020EE4B6
:10578400F02290020EE4F0222290020EE0FFEFD30A
:0F5794009404400A90020EE4F090020FE4F02219
:103A6200900220E0FFEF702A90020EE0FFEFD39465
:103A7200024003023E9E306303023E9E2061030227
:103A82003E9E90021FE0FF900220EFF0900221E4A0
:103A9200F022900220E0FFEFB40117900223E0FE33
:103AA200A3E0FFEE4420FE129307C261900220E4DD
:103AB200F022900220E0FFEF64027052900221E0B7
:103AC200FFEF701D306303023E9E900223E0FEA3CF
:103AD200E0FFEE4440FE129307900221E004F02240
:103AE20022900221E0FFEFB4011E306303023E9EEA
:103AF200900225E0FEA3E0FF129307C2619002202C
:103B0200E4F0900221E4F022900220E4F0229002FC
:103B120020E0FFEF64037072900221E0FFEF701C5F
:103B2200306303023E9E900223E0FEA3E0FFEE44D8
:103B320060FE129307900221E004F022900221E03D
:103B4200FFEFB40118306303023E9E900225E0FEAF
:103B5200A3E0FF129307900221E004F022900221D9
:103B6200E0FFEFB4021E306303023E9E900227E0A4
:103B7200FEA3E0FF129307C261900220E4F09002DC
:103B820021E4F022900220E4F022900220E0FFEFF4
:103B920064046003023D2B900221E0FFEF7033903A
:103BA2000223E0FEA3E0FF900225E0FCA3E0FD1269
:103BB2008B1F90022BE4F0A3E4F090022DE4F0A31B
:103BC2007480F0900229E4F0A3E4F0900221E00472
:103BD200F022900221E0FFEFB4011C306303023EA9
:103BE2009E900223E0FEA3E0FFEE4480FE129307C4
:103BF200900221E004F022900221E0FFEFB40218CB
:103C0200306303023E9E900225E0FEA3E0FF129382
:103C120007900221E004F022900221E0FFEF64030A
:103C22007063306303023E9E900229E475F0011234
:103C32008560AFF0FEEF25E0FFEE33FE74002FF556
:103C42008274043EF583E0F569A3E0F56AAF6AAEDB
:103C52006912930790022CE0256AF090022BE0355E
:103C620069F090022EE024FFF090022DE034FFF084
:103C720090022DE0FEA3E0FFEF4E600222229002AE
:103C820021E004F022900221E0FFEFB4041E306331
:103C920003023E9E90022BE0FEA3E0FF12930790E8
:103CA20002227464F0900221E004F022900221E0EA
:103CB200FFEF6405706D900222E0FFEF7019900231
:103CC20030E004F0700690022FE004F0900220E44D
:103CD200F0900221E4F022206403023E9EC2648539
:103CE200316B85326C900221E4F0E56CB40011E591
:103CF2006BB4900C900220E4F0900221E4F0C261D7
:103D0200E56C64017004E56B64906003023E9E9072
:103D12000221E4F0900230E004F0700690022FE0FD
:103D220004F022900220E4F022900220E0FFEF64EF
:103D3200056003023E94900221E0FFEF702B900297
:103D42002BE4F0A3E4F090022D7402F0A3E4F090CF
:103D52000229E4F0A3E4F0900223E0FEA3E0FF12C4
:103D62008576900221E004F022900221E0FFEFB478
:103D7200011C306303023E9E900223E0FEA3E0FF9B
:103D8200EE44A0FE129307900221E004F02290027A
:103D920021E0FFEF64027063306303023E9E9002F3
:103DA20029E475F001128560AFF0FEEF25E0FFEE29
:103DB20033FE74002FF58274043EF583E0F569A3A7
:103DC200E0F56AAF6AAE6912930790022CE0256AA9
:103DD200F090022BE03569F090022EE024FFF09083
:103DE200022DE034FFF090022DE0FEA3E0FFEF4E43
:103DF20060022222900221E004F022900221E0FFE0
:103E0200EFB4031E306303023E9E90022BE0FEA33A
:103E1200E0FF1293079002227464F0900221E00402
:103E2200F022900221E0FFEF64047060900222E031
:103E3200FFEF7014900230E004F0700690022FE061
:103E420004F0900221E4F022306451C26485316BA7
:103E520085326C900221E4F0E56CB40011E56BB49C
:103E6200900C900220E4F0900221E4F0C261E56C33
:103E7200B40129E56BB49024900230E004F070069E
:103E820090022FE004F0900221E4F022900220E45C
:0C3E9200F022900221E4F0900220E4F005
:013E9E002201
:047999008E0F8F10AE
:10799D00D3E510947DE50F940040047F0180027FB4
:1079AD0000C3E510943FE50F940050047E01800262
:1079BD007E00EE4FFFEF6003027A95E510AE0F7873
:1079CD0002C333CE33CED8F9FF745B2FF582745DCD
:1079DD003EF583E493F511740193F512E510AE0FA6
:1079ED007802C333CE33CED8F9FF74592FF5827494
:1079FD005D3EF583E493FE740193FF8F1790020EA5
:107A0D00E0FFEF6405FF90024DEFF090020FE0FFF5
:107A1D00EF6401FF90024EEFF0AD12AC11AF1712F3
:107A2D008DD190020EE0FFEF6405FF90024DEFF057
:107A3D0090020FE0FFEF6403FF90024EEFF075151B
:107A4D0000751600C3E51594045033AE15AF1674CA
:107A5D00002FF58274043EF583E0FF7E008E138FB8
:107A6D0014AB14AD12AC11AF17128C4B0512E512FD
:107A7D00700205110516E5167002051580C69002F7
:087A8D004DE4F090024EE4F01C
:017A950022CE
:109084008E188F197B017A047900AC02AD01AF19F7
:10909400AE18127215E5192480FFE5183400FE7B22
:0D90A400017A047980AC02AD011272152230
:048576008E588F5933
:10857A00E559AE587802C333CE33CED8F9FF745BCF
:10858A002FF582745D3EF583E493F55A740193F5F1
:10859A005BE559AE587802C333CE33CED8F9FF74AF
:1085AA00592FF582745D3EF583E493FE740193FFBF
:1085BA008F5E755C00755D00C3E55C9404502BAD5D
:1085CA005BAC5AAF5E1291E9AC5CAD5D74002DF5FF
:1085DA008274043CF583EFF0055BE55B7002055A93
:0A85EA00055DE55D7002055C80CEC2
:0185F4002264
:088B1F008E5F8F608C618D6296
:108B2700756300756400E5602401FFE55F3400FEAE
:108B3700EF25E0FFEE33FEC3E5649FE5639E502912
:108B47000562E562AE617002056114FF1271BEAC89
:108B570063AD6474002DF58274043CF583EFF00572
:098B670064E5647002056380BD41
:018B700022E2
:109307008E1D8F1E2063FD851D25851E26750C006D
:03931700D26322FC
:10680A00206203026970C262900210E0FFEF600327
:10681A00026901900217E0FEA3E0FFEFB4FF22EE47
:10682A00B41F1E7BFF7A5D7948128F629000037451
:10683A000AF0900003E0FFEF70F875840075EF032B
:10684A0022900217E0FEA3E0FFEEFF7E008F779012
:10685A000218E0FFEF54FFF578E57770107FFF8F9D
:10686A0078900245E4F09002487401F022E577B48A
:10687A001521E578C39433501A9002457401F090BB
:10688A000247E578F09001F77401F0900247E0FFC3
:10689A008F4122E577B41624E578C39472501D908F
:1068AA0002457402F0900247E578F09001F774020D
:1068BA00F0900247E0FF9001F9EFF022E577D394D8
:1068CA00004034E577C39415502DE578D394004001
:1068DA0026E578C394FB501F9002457403F090019B
:1068EA00EAE577F09001EBE578F0900246E577F07B
:1068FA00900247E578F022900210E0FFEF64027000
:10690A0065900217E0FEA3E0FFEF64014E70299044
:10691A000220E0FFEF70F8900223E4F0A3747FF006
:10692A0090021BE0FEA3E0FF900225EEF0A3EFF039
:10693A0090021F7404F0D261900217E0FEA3E0FFF8
:10694A00EF64024E7020900220E0FFEF70F8900290
:10695A001BE0FEA3E0FF900223EEF0A3EFF090020B
:06696A001F7405F0D2616C
:016970002204
:10FC0000C2AF12FCD812FD10E4F552F553E42553AF
:10FC1000FFE5523480FE12FCB6AD07AF53AE521270
:10FC2000FC5F0553E55370020552C3E552948040D2
:10FC3000DC755280755300AF53AE5212FCC7AD074E
:10FC4000AF53AE5212FC8A0553E55370020552C3FE
:10FC5000E55294F440E1D2AF75840075EF0122C201
:10FC6000AF75840F53A1FEE4F5B1F58443B701F5F8
:10FC700084438F018E658F668F828E83EDF0E4F56D
:10FC800084538FFEF58453B7FE22C2AF75840F53A1
:10FC9000A1FE75B110E4F58443B701F584438F01EB
:10FCA0008E658F668F828E83EDF0E4F584538FFE30
:10FCB000F58453B7FE22C2AF75B1218E678F688F6E
:10FCC000828E83E493FF22C2AF75B1318E678F6855
:10FCD0008F828E83E493FF22C2AFE4FFFEE4F5B18E
:10FCE000F58443B701F584758F03AD07AC068C65C9
:10FCF0008D668D828C83F0F58FF58453B7FE2FFFD0
:10FD000074043EFEC3948040D4E4F58453B7FE22CD
:10FD1000C2AF7F007E8075B110E4F58443B701F572
:04FD200084758F0354
:10FD2400AD07AC068C658D668D828C83F0F58FF5FE
:10FD34008453B7FE2FFF74043EFEC3648094744062
:08FD4400D1E4F58453B7FE225F
:101BF800C0D0C000C001C083C082C0E0C0F0C00730
:101C0800A291305001B37829E233F208E233F208A6
:101C1800E233F208E233F208E233F208E233F20880
:101C2800E233F208E233F208E233F208E233F20870
:101C3800E233F208E233F208E233F208E233F20860
:101C4800E233F208E233F208E233F208E233F20850
:101C5800E233F208E233F208E233F208E233F20840
:101C6800E233F208E233F208E233F208E233F20830
:101C7800E233F208E233F208E233F208E233F20820
:101C8800E233F208E233F208E233F208E233F20810
:011C9800E269
:101C990033F208E233F208E233F208E233F208E2FF
:101CA90033F208E233F2305C3A90217F7850E2183F
:101CB900203C03936028E218937023E21893601E76
:101CC900E218937019E218936014E21893600FE216
:101CD9001893700AE218937005E218936011C24BC9
:101CE900204C07C24BC24C021F58C24C021F2E90F7
:101CF90027CF78507F00E218203C03932FFFE2188A
:101D0900932FFFE218932FFFE218932FFFE2189306
:101D19002FFFE218932FFFE218932FFFE218932F5A
:101D2900FFE218932FFF90217F754200E218931369
:101D390092475003754238752200E21893139214A2
:101D4900500363421CE21893139213500363420E2B
:0C1D5900E218931392125003634246E21A
:101D650018931392115003634223E21893139210B0
:101D75008522435003634251752200E21893139262
:101D8500145003634268E21893139213500363429D
:101D950075E21893139212500363427AE218931373
:101DA5009211500363423DE2189313921085224429
:101DB500500363421F752200E218931392175003D4
:101DC50063424FE218931392165003634226E218BA
:101DD500931392155003634252E2189313921450D1
:101DE50003634229E218931392135003634215E2E9
:101DF5001893139212500363420BE2189313921136
:101E05005003634245E2189313921085224550030F
:101E1500634262E218931392145003634231E2184D
:101E2500931392135003634219E2189313921250BD
:101E35000363420DE218931392115003634207E2C4
:101E4500189313921085224650036342437522006E
:041E5500E2189313E9
:101E59009216E21893139215E21893139214E2184A
:101E690093139213E21893139212E2189313921197
:101E7900E21893139210852247E54765427025A21F
:101E8900479248E543900051F0E544900052F0E54F
:101E990045900053F0E546900054F0D24AC24BC237
:101EA9004C021F5823F89026D093F99026CFE89337
:101EB900602EB40104B2478027B40205E86243806A
:101EC9001FB40305E862448017B40405E86245803D
:101ED9000FB40505E862468007C24B304C71804556
:101EE900204B04D24B801B204C0DD24C90005AE061
:101EF900B50700400D805890005AE0B50700400230
:101F0900802390005AEFF0A2479259900056E5437A
:101F1900F0900057E544F0900058E545F0900059DD
:101F2900E546F0802AA2599248900056E090005167
:101F3900F0900057E0900052F0900058E090005364
:101F4900F0900059E0900054F0D24AC24BC24C12B2
:101F59001F6CD007D0F0D0E0D082D083D001D00060
:071F6900D0D022C0D0C0005F
:101F7000C0E0303F4EE554B40833A242B392B37888
:101F80007EE66036167883E6A2E7304401B39242DB
:101F900092B2A2E7787FE633F67880E633F678816E
:101FA000E633F67882E633F67883E633F6D55403E3
:101FB000755408D0E0D000D0D022C257D0E0D00075
:101FC000D0D022D0E0D000D0D022C0D0C000C001FC
:101FD000C083C082C0E0C0F0A291204F01B378114D
:101FE000E213F208E213F208E213F208E213F20835
:101FF000E213F208E213F208E213F208E213F20825
:10200000E213F208E213F208E213F208E213F20814
:10201000E213F208E213F208E213F208E213F20804
:10202000E213F208E213F208E213F208E213F208F4
:05203000E213F208E2DA
:1020350013F208E213F290217F7811E208931392CC
:102045000FE2089313920EE2089313920DE20893A0
:1020550013920CE2089313920BE2089313920AE28F
:102065000893139209E20893139208852148E20820
:102075009313920FE2089313920EE2089313920DB5
:10208500E2089313920CE2089313920BE208931360
:10209500920AE20893139209E208931392088521A4
:1020A50049E2089313920FE2089313920EE2089304
:1020B50013920DE2089313920CE2089313920BE22C
:1020C500089313920AE20893139209C20885214ADC
:1020D500305C3DE5489024CF854921300E020583CB
:1020E50093602D14F875F003A49023802582F58262
:0B20F500E5F03583F583E493F9A3E4E4
:102100009390227F654A93C965499329B401005091
:10211000048836D241122127D0F0D0E0D082D0837B
:10212000D001D000D0D022303D27C392B27884169F
:10213000E6701E76087887E6A2E1304501B392B3D7
:10214000A2E17885E613F67886E613F67887E6133B
:10215000F622EF90237F75F003A42582F582E583B4
:1021600035F0F583C23D7400937885F67401937859
:1021700086F67402937887F6C23FC23ED23D2200B3
:10218000000000000000000000000000000000004F
:10219000000000000000000000000000000101003D
:1021A000000000000000000000000000000001002E
:1021B0000000000000000100000001010101010019
:1021C000000000000000000000000000000001000E
:1021D00000000000000000000000000001010100FC
:1021E00000000000000001000000010000010100EB
:1021F00000000100010101010101010101010100D3
:1022000000000000000000000000000000000100CD
:1022100000000000000001000000010001010100B9
:1022200000000000000001000000010001010100A9
:102230000000010001010100010101010101010093
:102240000000000000000100000001000101010089
:102250000000010001010100010101010101010073
:102260000000010001010100010101010101010063
:102270000000010101010101010101010101010051
:10228000010102010202030102020302030304012D
:102290000202030203030402030303030304050110
:1022A00002020302030304020303040304040502FD
:1022B00003030403040405030404040405050601E0
:1022C00002020302030304020303030304040502DE
:1022D00003030403030405030404050405050602BF
:1022E00003030403040405030404050405050603AD
:1022F0000404050405050604050506050606070190
:10230000020203020303040203030403040405029C
:10231000030304030404050304040504050506027D
:10232000030304030404050304040504050506036C
:10233000040405040505060405050605060607024E
:10234000030304030404050304040504050506034C
:10235000040405040505060405050605060607032D
:10236000040405040505060405050605060607041C
:10237000050506050606070506060706070708FD04
:10238000D00C73700E3CF01AAF101E7F9022EC70D0
:1023900026D6F02ACBB02CA3F032BEB03417D03CF6
:1023A000B6D0461FB04E77F050F950526AB056DEA4
:1023B0009058BA306ACF3072D270745CD076E8F040
:1023C000786BD098E5709AF8309CBB50A40F70AA37
:1023D0007A70B26730B45DB0B8FCB0C26F50C65509
:1023E000D0CA3D90D489B0DA94F0DCD790E463B0E1
:1023F000EA0BF0F43170F8DD310AB571148FF11881
:10240000D1D126EB512AF6112C8B71463F5148B1A0
:10241000F14AACB14CC4F152D9B1546D915A2EF17C
:1024200062BD116687916A9AD16CF29172D551782A
:1024300019F18C71B192D8D19A32D1AA47D1B25A3E
:1024400091B452F1C67531CC1D71D2A951DCD0B115
:10245000E85E11EA2B11F2EED212F392147D3216DD
:10246000973226D8B232C5F234F7124AEA524C9F5C
:0D2470005254A5D2582B725A7552644FD2A7
:10247D0068C1726ADC326C78D2865F128C83729C72
:10248D004EB2A66972AC1C72B433D2CC18F2EABB50
:10249D00330CCE33141EB32803F32EE51332F85349
:1024AD003498735848F36472736845738617B39400
:1024BD007313A63C93B221D3B41B53B829B3C641B1
:1024CD00F3D8000000000000000000000000000034
:1024DD000000000000000000006A00000000000085
:1024ED00620D0000000000000000006F00480000B9
:1024FD0000000000000000000000000000006C2241
:10250D0000000000000000000000000000000000BE
:10251D005B00000000000000000000004100001EF4
:10252D004759000000260000001D00001000003576
:10253D000000003D006B0043000000000000004B58
:10254D00000500000000000000380023000000001E
:10255D000000000000000000004C00000000000022
:10256D00000000000000000000000000000032002C
:10257D0000040000000000000000000012600037A1
:10258D000A0000000000000000000000000800002C
:10259D00611346000000000000254D34000057294E
:1025AD0011000000000000640000000000000000A9
:1025BD00000000003A4A00002E4F190000001F00D5
:1025CD000000000000630000000000000027000074
:1025DD00001B000000000000000B5F3C006E5D441E
:1025ED000000006D0000000000000000005300001E
:1025FD00360000283F5E00000000000000000300D0
:10260D00003000700000006900406700000000000D
:10261D0000550000420000210000000000001500E0
:10262D0000000000000000000000005C001700002A
:10263D000020000068020054000E58001C0000002D
:10264D0000000000005A000000000000002F0000F4
:10265D00002B00000000240000006600390000007F
:10266D00005100000009005200000045000000006C
:10267D00000000310000002A0C000000001A0000CC
:10268D00000000560000334E000000000000000066
:10269D000000002C1400003B07003E00000000006D
:1026AD00000000000000001800001600502D06006C
:1026BD0049000000000000000000650F000000014F
:1026CD0000000000000000000600000006000600EB
:1026DD0005020600060006000404060005040208B3
:1026ED0006000000060006000600060004080600AD
:1026FD00060006000508060006000210060006008A
:10270D000301000006000600020206000600044058
:10271D00060006000410060006000600060006006E
:10272D00060006000510060006000600060006005D
:10273D000600010106000600060006000302060061
:10274D000600000006000600050106000402020452
:10275D00060006000600060006000600060006003C
:10276D000480060002010420060006000600060093
:10277D00060006000600060006000600060006001C
:10278D00060006000600040106000600060006000D
:10279D0006000310060006000600060006000600EF
:1027AD0006000600060006000600060003080600E7
:1027BD0006000600060003040600060006000600DB
:1027CD0006000002020402040406020404060406C4
:1027DD000608020404060406060804060608060890
:0D27ED000806020404060406060804060699
:1027FA000806080806040606080608080606080861
:10280A000608060604020404060406060804060668
:10281A000806080806040606080608080606080840
:10282A000608060604040606080608080606080836
:10283A000608060604060808060806060408060628
:10284A000406040402020404060406060804060632
:10285A000806080806040606080608080606080800
:10286A0006080606040406060806080806060808F6
:10287A0006080606040608080608060604080606E8
:10288A0004060404020406060806080806060808E0
:10289A0006080606040608080608060604080606C8
:1028AA0004060404020608080608060604080606C2
:1028BA0004060404020806060406040402060404C4
:0528CA000204020201FE
:03000000029369FF
:0C936900787FE4F6D8FD7581A1025F5901
:1084F600BB010689828A83E0225002E722BBFE0284
:09850600E32289828A83E49322B6
:10850F00BB010CE58229F582E5833AF583E0225021
:10851F0006E92582F8E622BBFE06E92582F8E2226B
:0D852F00E58229F582E5833AF583E4932285
:10853C00BB010689828A83F0225002F722BBFE011E
:02854C00F32218
:10854E00EF8DF0A4A8F0CF8CF0A428CE8DF0A42E41
:02855E00FE22FB
:10856000A3F8E0C5F025F0F0E582158270021583CE
:06857000E0C838F0E8222B
:00000001FF
